:100000000C9446000C94A0210C94952218950000A5
:10001000189500001895000018950000189500002C
:10002000189500001895000018950000189500001C
:10003000189500000C94E420189500001895000015
:1000400018950000189500000C943A2418950000AB
:1000500018950000189500001895000018950000EC
:1000600018950000189500001895000018950000DC
:1000700018950000189500001895000018950000CC
:100080000C94422118950000189500008FEF8DBF49
:10009000C0E8E8E94E2E80E48EBFD0E4FFE35F2E97
:1000A000A89584B7082E877F84BF88E1992780931D
:1000B000600090936000EEEFFFE3A0E0B1E08827DE
:1000C0008D933197E9F787E68093C40080E08093B1
:1000D000C50088E18093C1006624E6EDF5E60E9444
:1000E000F8310E94C3250E94CA253E9A469A7DB5E2
:1000F00071607DBD0E942E260E94E526A5E0B1E03C
:100100009C930B9813980F9A3F9A52985398559A2C
:10011000569A579A209854985C9AE89AE99A70915E
:100120006E00716070936E0017985D98479884E038
:1001300085BD80E084BD70916E00716070936E002B
:1001400084E085BD80E08093800089E08093810019
:1001500070916F007D7F70936F0085ED92E09093BA
:1001600089008093880080918100887F809381003E
:10017000579A569A81E08093B10081EF8093B00046
:1001800088278093B10080E08093900089E080937D
:100190009100709171007D7F7093710085ED92E008
:1001A000909399008093980080919100887F80932C
:1001B000910087E880937A0080EC80937C00E2EEE7
:1001C000F5E60E94F8310E94C3250E94D71FEAED90
:1001D000FEE0A1E9BFE00E941B32E1E9FFE0A0E8F8
:1001E000BFE31127222703E032E00E94B4310E94CE
:1001F000BB25E6EFF5E60E94F8310E94C3250E9478
:10020000CA25EAEFF5E60E94F8310E94C32580E096
:1002100080931A0AE1E0F0E007B7096007BFC895CC
:100220000092190A0091190A0F3F11F40C941D0154
:10023000AAE1BAE08C9182608C93E2E0F0E007B72B
:10024000096007BFC8950092190A0091190A0D3F6D
:1002500011F40C943001AAE1BAE08C9184608C9383
:10026000E3E0F0E007B7096007BFC8950092190AFC
:100270000091190A003D81E009F480E08F9300911C
:10028000190A003C81E009F480E09F9189238823CA
:1002900011F40C945001AAE1BAE08C9188608C931F
:1002A000E4E0F0E007B7096007BFC8950092190ABB
:1002B0000091190A073D11F40C946301AAE1BAE018
:1002C0008C9180618C9300911A0A003011F00C948B
:1002D0007301EEE0F6E60E94F8310E94C3250E9409
:1002E000CA250C948A0117985D9AE2E1F6E60E940D
:1002F000F8310E94C325EAE1FAE0A0E8BFE30E94DA
:100300002B320E94BB250E94CA2584EC99E00E94F2
:1003100085265D98EAE1F6E60E94F8310E94C32541
:100320000E94CA25E1E0F0E0ABE1BAE091E00E9472
:10033000BE3200911B0A053010F40C94A20180E03B
:1003400080931B0A00911B0A013081E009F080E0D4
:100350008F9300911B0A043081E009F080E09F91A7
:10036000892B882311F40C94B601E898E2E0F0E0C0
:10037000ACE1BAE091E00E94BE3200911C0A033069
:1003800010F40C94C60181E080931C0AE3E0F0E0D5
:10039000AEE1BAE091E00E94BE3200911E0A023046
:1003A00010F40C94D60181E080931E0AE4E0F0E0A2
:1003B000AFE1BAE091E00E94BE3200911F0A023024
:1003C00010F40C94E60181E080931F0AE5E0F0E070
:1003D000A0E2BAE091E00E94BE320091200A033010
:1003E00010F40C94F60181E08093200AE6E0F0E03E
:1003F000A1E2BAE091E00E94BE320091210A0230EF
:1004000081E008F480E08F9300911B0A013081E0C5
:1004100009F080E09F91892B8F9300911B0A043093
:1004200081E009F080E09F91892B882311F40C94DE
:100430001C0280E08093210AE7E0F0E0A2E2BAE04B
:1004400091E00E94BE320091220A023010F40C9416
:100450002C0280E08093220AE8E0F0E0A3E2BAE018
:1004600091E00E94BE320091230A083281E008F038
:1004700080E08F930091230A073380E010F009F0A9
:1004800081E09F91892B882311F40C944A0282E326
:100490008093230AA3E2BAE00D9111274AE050E0CD
:1004A0000E943E31A4E2BAE00D931C93A4E2BAE0AC
:1004B0000D911C91065F1F4FA6E2BAE00D931C93AD
:1004C000E9E0F0E0A8E2BAE091E00E94BE320091DB
:1004D000280A003011F00C9472028AE08093900F89
:1004E0000C949002013011F00C947B0284E1809313
:1004F000900F0C949002023011F00C9484028EE163
:100500008093900F0C949002033011F00C948D02A4
:100510008CE38093900F0C9490028AE08093900F6C
:10052000EAE0F0E0ABE2BAE091E00E94BE32009176
:100530002B0A0A3081E008F080E08F9300912B0AAB
:10054000063980E010F009F081E09F91892B882323
:1005500011F40C94AE0284E680932B0AEBE0F0E0F9
:10056000AAE2BAE091E00E94BE3200912A0A00306D
:1005700081E008F080E08F9300912A0A043680E041
:1005800010F009F081E09F91892B882311F40C94DD
:10059000CC0280E080932A0AECE0F0E0A8E3BAE025
:1005A00091E00E94BE320091380A043081E009F0E7
:1005B00080E08F930091380A073081E008F480E0F2
:1005C0009F91892B882311F40C94E90281E0809398
:1005D000380A0091380A003011F00C94F20284E0DD
:1005E00080938B0F0091380A013011F00C94FB02BC
:1005F00083E080938B0F0091380A023011F00C9445
:10060000040382E080938B0F0091380A033011F0CD
:100610000C940D0381E080938B0FEDE0F0E0A9E2F4
:10062000BAE091E00E94BE320091290A023010F433
:100630000C941D0381E08093290AE0E1F0E0ABE334
:10064000BAE091E00E94BE32E1E1F0E0ACE3BAE052
:1006500091E00E94BE32E2E1F0E0ADE2BAE091E06A
:100660000E94BE3200912D0A033010F40C943B031B
:1006700080E080932D0AE3E1F0E0AEE2BAE091E0A1
:100680000E94BE3200912E0A033010F40C944B03EA
:1006900080E080932E0AE0E2F0E0ACE2BAE091E084
:1006A0000E94BE3200912C0A023010F40C945B03BD
:1006B00080E080932C0AAAE2BAE00D91112747E06E
:1006C00050E00E943E31A4E3BAE00D931C9305ED87
:1006D00012E0A4E3BAE04D915C91040F151FA4E36E
:1006E000BAE00D931C93ABE2BAE00D91112742E002
:1006F00050E00E943E31A6E3BAE00D931C9305ED55
:1007000012E0A6E3BAE04D915C91041B150BA6E341
:10071000BAE00D931C93A6E3BAE00D911C91A4E3FB
:10072000BAE04D915C91041B150BA0E7BFE00D935F
:100730001C9300912C0A003011F00C94AD03A0E73B
:10074000BFE00D911C9144E150E00E947A25A0E7A2
:10075000BFE04D935C930C94B903A0E7BFE00D910B
:100760001C9148E250E00E947A25A0E7BFE04D933B
:100770005C93A0E7BFE00D911C914AE750E00E9416
:100780003E31A2E7BFE00D931C93A6E3BAE00D91C2
:100790001C91A2E7BFE04D915C91041B150BA2E7F1
:1007A000BFE00D931C93A6E3BAE00D911C91A4E366
:1007B000BAE04D915C91041B150BA8E7BFE00D93C7
:1007C0001C93A8E7BFE00D911C9148E250E00E9405
:1007D0007A25A8E7BFE04D935C93E2E2F0E0ADEA52
:1007E000BFE091E00E94BE320091AD0F023010F4E4
:1007F0000C94FD0380E08093AD0FE3E2F0E0AFE204
:10080000BAE091E00E94BE3200912F0A043010F449
:100810000C940D0481E080932F0AE4E2F0E0A2E35F
:10082000BAE091E00E94BE320091320A003110F429
:100830000C941D0480E08093320AE5E2F0E0A3E32B
:10084000BAE091E00E94BE320091330A003110F408
:100850000C942D0480E08093330AE6E2F0E0A0E3FC
:10086000BAE091E00E94BE320091300A003110F4EB
:100870000C943D0480E08093300AE7E2F0E0A1E3CD
:10088000BAE091E00E94BE320091310A003110F4CA
:100890000C944D0480E08093310AE8E2F0E0A5EB8F
:1008A000BFE091E00E94BE320091B50F023010F41B
:1008B0000C945D0480E08093B50FE9E2F0E0A4EBD6
:1008C000BFE091E00E94BE320091B40F023010F4FC
:1008D0000C946D0480E08093B40FECE2F0E0ACED9A
:1008E000BEE092E00E94BE32ACEDBEE00D911C91E4
:1008F000023E5FEF150780E00CF481E08F93ACEDD2
:10090000BEE00D911C910E3150E0150780E014F00F
:1009100009F081E09F91892B882311F40C949404B1
:10092000ACEDBEE00E94A631EFE2F0E0A1E4BAE057
:1009300091E00E94BE328BE58093A90F81E68093FF
:10094000AA0F8BE58093AB0F81E68093AC0F88E50F
:100950008093430A8AE58093440A84E68093450A9B
:1009600082E68093460A88E58093470A8AE5809369
:10097000480A84E68093490A82E680934A0A8EE513
:100980008093B20F8EE58093B30F78940091660048
:100990004BE1041BA2E4BAE00C934091420A00919F
:1009A000410A041711F40C94EB0480E880B984EF39
:1009B00091E00E94852680E289B984EF91E00E944F
:1009C00085260091BA0F003411F00C94E9040C94C0
:1009D000F21C0C94D5040E94FE240091000100300A
:1009E00011F00C941B06E8E3F6E60E94F8310E9431
:1009F000C3250E94CA2580E08093E70E80E880B975
:100A00008AEF90E00E9485260E94D71F0091BA0FBE
:100A1000003411F00C940E050C94F21C0091E70EBA
:100A20000A3018F011F00C949B050091B60F0F3F9F
:100A300081E009F080E08F930091B00F083881E0E9
:100A400008F480E09F9189238F930091B70F0F3FA7
:100A500081E009F080E09F9189238F930091B10F8D
:100A6000083881E008F480E09F918923882311F4FD
:100A70000C944105A7EEBEE08C918F5F8C930C9493
:100A8000440580E08093E70E0091E70E0A3011F0F4
:100A90000C949B05ACEDBEE00E94A631ACEBBFE030
:100AA0000E94A63181E08093E60E0091E60E0530AB
:100AB00018F011F00C9478050E94D71FACEBBFE042
:100AC0000D911C91AAEDBEE04D915C91040F151F94
:100AD000ACEBBFE00D931C938AE090E00E9485266A
:100AE000A6EEBEE08C918F5F8C9310F40C945505AC
:100AF000ACEBBFE00D911C9145E050E00E947A25DF
:100B0000ACEBBFE04D935C9300EF11E0ACEBBFE0CA
:100B10004D915C91041B150BACEBBFE00D931C9346
:100B20000E94DB2080E08093B60F80E08093B70FB7
:100B30008BE08093E70E0091E70E0B3010F40C94DD
:100B400019060091B60F0F3F81E009F080E08F9306
:100B50000091B00F083881E008F480E09F9189236C
:100B60008F930091B70F0F3F81E009F080E09F91D4
:100B700089238F930091B10F083881E008F480E059
:100B80009F918923882311F40C94CD05A7EEBEE034
:100B90008C918F5F8C930C94D0058BE08093E70E43
:100BA0000091E70E053111F00C94190680E0809356
:100BB000B60F80E08093B70FACEBBFE00D911C91B6
:100BC000023E5FEF150780E014F009F081E08F939B
:100BD000ACEBBFE00D911C910E3150E0150780E0A9
:100BE0000CF481E09F918923882311F40C94100662
:100BF000ECE2F0E0ACEBBFE092E07BE70E94AD32CC
:100C00000E94DB208AEF90E00E9485260E94DB2074
:100C10008AEF90E00E9485260C944C1F0C941906D4
:100C200080E08093E70E5D9A88EE93E00E9485262F
:100C30005D980C94FE0400910401003011F00C94B6
:100C40004306E4E5F6E60E94F8310E94C325E4E09D
:100C5000F1E0A0E8BFE30E942B320E94BB250E9476
:100C6000CA2580E880B984EF91E00E9485260E9421
:100C7000D71F0091BA0F003411F00C9441060C9468
:100C8000F21C0C943106179AEAE6F6E60E94F83157
:100C90000E94C3250E94CA25ABE4BAE0EEE7F6E65F
:100CA0000E94F8310E946B31ABE4BAE0E0E1F0E081
:100CB0000E94322A40E050E060E070E00E9408327A
:100CC0001CF011F00C9466060C9468060C9400F06D
:100CD000ECE8F6E60E94F8310E94C3250E94CA257E
:100CE000ABE4BAE0E2EAF6E60E94F8310E946B312A
:100CF000ABE4BAE0E0E1F0E00E94322A40E050E0EC
:100D000060E070E00E9408321CF011F00C948A063A
:100D10000C945B078AE0ABE4BAE00E94AE29009134
:100D20000C01003011F00C94580740E850E08AE0C4
:100D3000A8E9B9E0E8940E941B2A009199090233BE
:100D400081E009F080E08F9300919A090E3281E0F2
:100D500009F080E09F9189238F9300919B090033D4
:100D600081E009F080E09F918923882311F40C949D
:100D7000580780E289B986E08093E60E0091E60E7E
:100D8000043618F011F00C9426070091E60E45E0A9
:100D9000041BA7EEBEE00C930091E70E0D3181E03D
:100DA00009F480E08F930091E70E0E3181E009F4A1
:100DB00080E09F9189238F930091E70E0F3181E0AE
:100DC00009F480E09F918923882311F40C941E0775
:100DD0000091E70E0C3281E009F480E08F930091DE
:100DE000E70E0D3281E009F480E09F91892388238A
:100DF00011F40C941E070091E70E0E3281E009F405
:100E000080E08F930091E70E0F3281E009F480E0DB
:100E10009F918923882311F40C941E07A7EEBEE04E
:100E2000EC91FF27A6EEBEE0AD90BB24A7E9B9E0A8
:100E3000AA0DBB1D91E07BE70E94AD32A6EEBEE09D
:100E40008C918F5F8C9310F40C94BE068AE00E9404
:100E5000DF29EEEAF6E60E94F8310E94C3250E94DF
:100E6000CA25ABE4BAE00E942F2D0E94832EABE48A
:100E7000BAE0ECECF6E60E94F8310E946B31ABE48C
:100E8000BAE0E0E1F0E00E94322A40E050E060E0A9
:100E900070E00E94083211F40C945407ABE4BAE0FD
:100EA0000E942F2D0E94832E0E945F1F0C944C1FC6
:100EB0008AE00E94DF29ABE4BAE0ECECF6E60E949F
:100EC000F8310E946B31ABE4BAE0E0E1F0E00E945F
:100ED000322A40E050E060E070E00E94083211F0F9
:100EE0000C94F5078AE0ABE4BAE00E94AE290091C9
:100EF0000C01003011F00C94E60783E08093180A8F
:100F0000E8948AE0A8E1BAE00E94F72982E3A8E128
:100F1000BAE08C93E8948AE0A8E1BAE00E94F7294D
:100F20008EE2A8E1BAE08C93E8948AE0A8E1BAE006
:100F30000E94F72980E3A8E1BAE08C93E8948AE064
:100F4000A8E1BAE00E94F7298FEF8093180AE8948D
:100F50008AE0A8E1BAE00E94F72981E08093E60EDA
:100F60000091E60E0F3518F011F00C94E607A6EE8E
:100F7000BEE0EC91FF27A8E1BAE091E00E94BE320A
:100F80000091E60E0E3281E009F080E08F9300912F
:100F9000E60E0F3281E009F080E09F91892B8823D3
:100FA00011F40C94D6078FEF8093180AE8948AE026
:100FB000A8E1BAE00E94F72980E289B9A6EEBEE076
:100FC0008C918F5F8C9310F40C94B0078AE00E9490
:100FD000DF29E8EDF6E60E94F8310E94C3250E9461
:100FE000CA250E945F1F47985D98E2EFF6E60E94CF
:100FF000F8310E94C32500911C0A003011F00C94B6
:101000000B08E4E0F7E60E94F8310E94C3250E9435
:10101000CA250C943308013011F00C941908EEE045
:10102000F7E60E94F8310E94C3250E94CA250C945D
:101030003308023011F00C942708E6E1F7E60E942D
:10104000F8310E94C3250E94CA250C94330803304E
:1010500011F00C943308EEE1F7E60E94F8310E949B
:10106000C3250E94CA2500911C0A003011F00C947F
:101070005F0880E08093D10E0091D00E0A3010F00E
:101080000C945D0882E390E00E948526A1EDBEE00D
:101090008C918F5F8C930091D10E043610F40C94D8
:1010A00053080C945D080091BA0F003411F00C94B1
:1010B0005B080C94F21C0C943C080C947F080130E3
:1010C00011F00C94690880E293E00E9485260C944C
:1010D0007F08023011F00C94730888E097E00E94BA
:1010E00085260C947F08033011F00C947F0888EE5D
:1010F00093E00E94852688E097E00E948526E6E23C
:10110000F7E60E94F8310E94C32580E08093CF0E5D
:1011100000912F0A003011F00C94340900911B0A41
:10112000013011F40C94E0080091B00F003081E020
:1011300009F480E08F930091B00F083581E008F446
:1011400080E09F9189238F930091B00F043681E056
:1011500010F009F080E09F918923882311F40C940A
:10116000DD080091B00F41E0041BA9EABFE00C9339
:101170000091B00F41E0040FAAEABFE00C93009188
:10118000B00F44E0041BA3E4BAE00C930091430ABF
:1011900042E0040FA4E4BAE00C930091B00F44E0E5
:1011A000040FA5E4BAE00C930091450A42E0041B49
:1011B000A6E4BAE00C930C94E00881E08093CF0E93
:1011C00000911B0A023011F00C9432090091B10F0A
:1011D000003081E009F480E08F930091B10F083571
:1011E00081E008F480E09F9189238F930091B10FF3
:1011F000043681E010F009F080E09F918923882374
:1012000011F40C942F090091B10F41E0041BABEADB
:10121000BFE00C930091B10F41E0040FACEABFE0D6
:101220000C930091B10F44E0041BA7E4BAE00C93C7
:101230000091470A42E0040FA8E4BAE00C93009141
:10124000B10F44E0040FA9E4BAE00C930091490AFD
:1012500042E0041BAAE4BAE00C930C94320981E04A
:101260008093CF0E0C948609013011F00C945E0926
:101270008CE58093A90F80E68093AA0F8CE580937C
:10128000AB0F80E68093AC0F89E58093430A8BE532
:101290008093440A83E68093450A81E68093460A58
:1012A00089E58093470A8BE58093480A83E680931B
:1012B000490A81E680934A0A0C948609033011F0AA
:1012C0000C9486098AE58093A90F82E68093AA0F81
:1012D0008AE58093AB0F82E68093AC0F87E580931D
:1012E000430A89E58093440A85E68093450A83E6AC
:1012F0008093460A87E58093470A89E58093480AE8
:1013000085E68093490A83E680934A0A0091AD0FEF
:10131000003011F40C94D80991E0A0E3BAE00E94E7
:10132000883106E54091300A041BA3E4BAE00C932F
:101330000091430A42E0040FA4E4BAE00C9391E068
:10134000A1E3BAE00E94883106E64091310A040F19
:10135000A5E4BAE00C930091450A42E0041BA6E420
:10136000BAE00C9391E0A2E3BAE00E94883106E56E
:101370004091320A041BA7E4BAE00C930091470A9B
:1013800042E0040FA8E4BAE00C9391E0A3E3BAE0D2
:101390000E94883106E64091330A040FA9E4BAE0BE
:1013A0000C930091490A42E0041BAAE4BAE00C93B2
:1013B00000911B0A023011F40C94130A0091B10F32
:1013C000003011F40C94100A0091B10F41E0041B9D
:1013D000ABEABFE00C930091B10F41E0040FACEA1F
:1013E000BFE00C930091B10F44E0041BA7E4BAE006
:1013F0000C930091470A42E0040FA8E4BAE00C9372
:101400000091B10F44E0040FA9E4BAE00C930091FD
:10141000490A42E0041BAAE4BAE00C930C94130AB4
:1014200081E08093CF0EEAE3F7E60E94F8310E9454
:10143000C325E1EBFFE0A0E8BFE30E942B320E944E
:10144000BB25E0E4F7E60E94F8310E94C325E0EBFB
:10145000FFE0A0E8BFE30E942B320E94BB25E6E438
:10146000F7E60E94F8310E94C3250E94CA25009128
:10147000CF0E003011F40C943D0A479880E0809321
:10148000B60F80E08093B70F84E690E00E94852637
:10149000E8E4F7E60E94F8310E94C32500911B0A98
:1014A000023011F40C94680A0E94C61B81E08093FC
:1014B000890F8091890F80938A0F0E9474190E946E
:1014C0008F1980E080939E0EA0E9BAE20E94A631B7
:1014D00000911F0A013011F00C94730A0E949B1FA7
:1014E0000E949B1F479800911E0A003011F00C9437
:1014F0007B0A17985D98E2E6F7E60E94F8310E94B1
:10150000C3250E94CA2580911E0A80931D0A80E08F
:1015100080937F0F80E08093860F80E080938F0F11
:1015200080E08093880F70E87093B30070E8709348
:10153000B400EEE7F7E60E94F8310E94C3250E944E
:10154000CA2500919C0E003011F00C94AB0A0E9449
:10155000010C0C94FF0B00919D0E003011F00C94C7
:10156000B50A0E94600C0C94FF0B0091A00E003095
:1015700011F00C94BF0A0E94BF0C0C94FF0B009159
:10158000A10E003011F00C94C90A0E94080D0C94B1
:10159000FF0B4C990C94F80A18990C94F80A479888
:1015A00070E87093B30070E87093B400809181008C
:1015B000887F8093810088278093B100809191007B
:1015C000887F8093910017985D98F89480E880B99F
:1015D0008AEF90E00E9485260091BA0F003411F046
:1015E0000C94F40A0C94F21C0E94D71F0C94E60A87
:1015F0000091BA0F003411F00C94000B0C94F21C03
:101600000E94D71F0091E20E003011F00C94A20B43
:1016100000911B0A013018F011F00C94110B0E947C
:10162000510D00911B0A033010F40C94190B0E9409
:101630005F100E94091200911B0A023011F00C94F5
:10164000230B0E94111600911B0A023011F00C941A
:10165000510B8AE00E94E829082F0F3F11F00C94EB
:10166000510B0091390A003011F00C94440B009199
:101670009E0E013011F00C94420B70916F007D7F33
:1016800070936F000C94510BA5ECBEE0E2EDF5E613
:101690000E94F8310E949E318AE0A5ECBEE00E94D3
:1016A000D2298BE00E94E829082F0F3F11F00C94FB
:1016B000790B00913A0A003011F00C946C0B0091F8
:1016C000A20E013011F00C946A0B709171007D7FB5
:1016D000709371000C94790BA9ECBEE0E2EDF5E695
:1016E0000E94F8310E949E318BE0A9ECBEE00E947E
:1016F000D2290091BB0F013011F00C94840B709132
:101700006F00726070936F000091BB0F023011F098
:101710000C948F0B70917100726070937100009146
:10172000BB0F033011F00C949F0B70916F0072602F
:1017300070936F007091710072607093710080E01F
:101740008093BB0FAFE6B0E00C9101FB81E00EF49B
:1017500080E08F93A1E7B0E00C9101FB81E00EF4F3
:1017600080E09F918923882311F40C94D30B00917E
:10177000E20E003011F00C94D10B479870E8709392
:10178000B30070E87093B40080918100887F8093EB
:10179000810088278093B10080919100887F809399
:1017A00091000C94FF0BAFE6B0E00C9101FB16F03A
:1017B0000C94DF0B89E0809381000C94E70B70E8B8
:1017C0007093B30080918100887F80938100A1E7AE
:1017D000B0E00C9101FB16F00C94F30B89E08093C0
:1017E00091000C94FB0B70E87093B4008091910011
:1017F000887F8093910081E08093B100479A0C9498
:10180000A10A40E054E08AE0A0E9BAE0E8940E942E
:101810001B2A8AE00E94E829082F0F3F11F00C9440
:10182000370C00911B0A023011F00C94270CA5EB29
:10183000BEE00D911C91A1ECBEE04D915C91041BAA
:10184000150BACE8BAE00D931C930C94350CADEA83
:10185000BEE00D911C91A9EBBEE04D915C91041B83
:10186000150BACE8BAE00D931C930C943D0C80E092
:1018700094E0ACE8BAE08D939C93ACE8BAE0AD900C
:10188000BD90AFE8BAE0AA0DBB1D0C91003011F07D
:101890000C945C0CACE8BAE0AD90BD90AEE8BAE058
:1018A000AA0DBB1D8C91ACE8BAE0AD90BD90AFE83D
:1018B000BAE0AA0DBB1D8C9381E080939C0E089525
:1018C00040E054E08AE0A0E9B2E1E8940E941B2ADB
:1018D0008AE00E94E829082F0F3F11F00C94960C23
:1018E00000911B0A023011F00C94860CA5EBBEE0AF
:1018F0000D911C91A1ECBEE04D915C91041B150B68
:10190000AEE8BAE00D931C930C94940CADEABEE0E3
:101910000D911C91A9EBBEE04D915C91041B150B40
:10192000AEE8BAE00D931C930C949C0C80E094E01C
:10193000AEE8BAE08D939C93AEE8BAE0AD90BD906E
:10194000AFE8B2E1AA0DBB1D0C91003011F00C9470
:10195000BB0CAEE8BAE0AD90BD90AEE8B2E1AA0D26
:10196000BB1D8C91AEE8BAE0AD90BD90AFE8B2E19E
:10197000AA0DBB1D8C9381E080939D0E089540E0DD
:1019800054E08BE0A0E9BAE1E8940E941B2A8BE0C6
:101990000E94E829082F0F3F11F00C94DF0CA1EBF7
:1019A000BEE00D911C91ADEBBEE04D915C91041B2E
:1019B000150BA0E9BEE00D931C930C94E50C80E0A0
:1019C00094E0A0E9BEE08D939C93A0E9BEE0AD90C9
:1019D000BD90AFE8BAE1AA0DBB1D0C91003011F02B
:1019E0000C94040DA0E9BEE0AD90BD90AEE8BAE164
:1019F000AA0DBB1D8C91A0E9BEE0AD90BD90AFE8F3
:101A0000BAE1AA0DBB1D8C9381E08093A00E0895CE
:101A100040E054E08BE0A0E9B2E2E8940E941B2A87
:101A20008BE00E94E829082F0F3F11F00C94280D3D
:101A3000A1EBBEE00D911C91ADEBBEE04D915C9130
:101A4000041B150BA2E9BEE00D931C930C942E0D04
:101A500080E094E0A2E9BEE08D939C93A2E9BEE011
:101A6000AD90BD90AFE8B2E2AA0DBB1D0C91003065
:101A700011F00C944D0DA2E9BEE0AD90BD90AEE822
:101A8000B2E2AA0DBB1D8C91A2E9BEE0AD90BD9063
:101A9000AFE8B2E2AA0DBB1D8C9381E08093A10E4A
:101AA00008950091B10F003011F00C94580D089575
:101AB00000912C0A003011F00C94110E0091890F46
:101AC000023011F40C94670D80E080938F0F4091E9
:101AD000900F00918F0F041710F40C94780D009163
:101AE000210A003011F00C94780D86E08093890F64
:101AF0004091470A0091B10F041781E010F009F0FE
:101B000080E08F934091490A0091B10F041781E062
:101B100008F480E09F91892B882311F40C94C50D63
:101B200081E08093810F0091210A003011F00C9424
:101B30009E0D70916F00726070936F0081E08093D2
:101B40008C0F00918D0F0A3781E008F480E08F93AD
:101B50000091290A003081E009F080E09F91892BF3
:101B6000882311F40C94C30D0091890F013011F4F6
:101B70000C94C30D0091890F063011F40C94C30D21
:101B800084E08093890F0C940F0E4091480A0091D5
:101B9000B10F041780E010F009F081E08F934091BD
:101BA0004A0A0091B10F041781E008F080E09F918C
:101BB0008923882311F40C940F0E80E080938C0FFE
:101BC00000918D0F0A3081E008F480E08F9300913E
:101BD0008D0F0A3781E010F009F080E09F91892392
:101BE000882311F40C94030E0091290A013011F09E
:101BF0000C94030E0091890F023011F00C94030E27
:101C000083E08093890F80E080938D0F0091890F8E
:101C1000043011F00C940F0E85E08093890F0C9422
:101C2000A20E0091890F023011F40C941A0E80E07C
:101C300080938F0F4091900F00918F0F041710F435
:101C40000C942B0E0091210A003011F00C942B0EF5
:101C500086E08093890F4091490A0091B10F0417E3
:101C600010F40C94680E81E08093810F0091210A9A
:101C7000003011F00C94410E70916F0072607093FF
:101C80006F0081E080938C0F00918D0F0A3781E007
:101C900008F480E08F930091290A003081E009F078
:101CA00080E09F91892B882311F40C94660E00919B
:101CB000890F013011F40C94660E0091890F0630E3
:101CC00011F40C94660E84E08093890F0C94A20E9C
:101CD00040914A0A0091B10F041710F00C94A20E23
:101CE00080E080938C0F00918D0F0A3081E008F422
:101CF00080E08F9300918D0F0A3781E010F009F09A
:101D000080E09F918923882311F40C94960E009112
:101D1000290A013011F00C94960E0091890F0230BF
:101D200011F00C94960E83E08093890F80E08093ED
:101D30008D0F0091890F043011F00C94A20E85E0F4
:101D40008093890F0091890F043011F00C94BD0F1E
:101D50004091470A0091B10F041781E010F009F09B
:101D600080E08F934091490A0091B10F041781E000
:101D700008F480E09F91892B882311F40C94BB0F09
:101D80004091470A0091B10F041718F011F00C941C
:101D9000E30E0EE510E0A1EBBFE04D915527041BCB
:101DA000150BA4E7BFE00D931C930EE510E0A4E72C
:101DB000BFE04D915C91040F151FA4E7BFE00D93A8
:101DC0001C930C94EB0EA1EBBFE08C91A4E7BFE059
:101DD0008D9388278C930091380A053018F011F004
:101DE0000C94620FA4E7BFE00D911C91A0E7BFE047
:101DF0004D915C910E943E31A4E7BFE00D931C938E
:101E0000A4E7BFE00D911C91A2E7BFE04D915C916A
:101E1000040F151FA4E7BFE00D931C93A4E7BFE0D8
:101E20000D911C91073751E015070CF402C00C947A
:101E30001F0F87E791E0A4E7BFE08D939C9300918B
:101E4000380A053011F40C94580F40918B0F009113
:101E5000400A041710F40C94560F80E08093400A57
:101E6000A4E7BFE04D915C91ADE3BAE00D911C9108
:101E7000041715071CF011F00C94400F0C944E0F32
:101E8000ADE3BAE00E946D25ADE3BAE08D919C917F
:101E900090938900809388000C94560FA4E7BFE0CC
:101EA0008D919C9190938900809388000C94600F91
:101EB000A4E7BFE08D919C91909389008093880066
:101EC0000C94BB0FA4E7BFE00D911C910656104087
:101ED000A4E7BFE00D931C93A4E7BFE00D911C9114
:101EE000A4E7BFE04D915C910E943E31A4E7BFE0C2
:101EF0000D931C93A4E7BFE00D911C91A8E7BFE0F0
:101F00004D915C910E943E31A4E7BFE00D931C937C
:101F1000A4E7BFE00D911C914AE050E00E947A25B1
:101F2000A4E7BFE04D935C93A4E7BFE00D911C9143
:101F3000A4E3BAE04D915C91040F151FA4E7BFE044
:101F40000D931C93A4E7BFE00D911C91073751E05E
:101F500015070CF402C00C94B30F87E791E0A4E7D7
:101F6000BFE08D939C93A4E7BFE08D919C919093EB
:101F70008900809388000C94E70FA6E7BFE08D915D
:101F80009C91909389008093880006E610E0A0E77A
:101F9000BFE04D915C910E943E31A4E7BFE00D93FC
:101FA0001C93A4E7BFE00D911C91A2E7BFE04D9107
:101FB0005C91040F151FA4E7BFE00D931C93A4E7E9
:101FC000BFE08D919C91ADE3BAE08D939C9300911D
:101FD000890F063011F40C9438108AE00E94E82929
:101FE000082F0F3F11F00C9436100091890F02302A
:101FF00081E009F080E08F930091890F043081E047
:1020000009F080E09F91892B882311F40C9417101C
:10201000A5ECBEE0E2EDF5E60E94F8310E949E31AB
:102020008AE0A5ECBEE00E94D2290C943610009103
:10203000890F013081E009F080E08F930091890FD2
:10204000053081E009F080E09F91892B882311F40D
:102050000C942D1082E08093890F0091890F03303A
:1020600011F00C94361085E08093890F0C944B107E
:102070008AE00E94E829082F0F3F11F00C944B10C2
:1020800070916F007D7F70936F0080E08093810F6F
:1020900081E08093890F4091890F00918A0F041786
:1020A00011F40C945E100E9474198AE00E94DF29DA
:1020B0000E948F198091890F80938A0F0895009153
:1020C000B10F003011F00C946610089500912C0AA5
:1020D000003011F00C9411110091890F023011F4AD
:1020E0000C94751080E080938F0F4091900F0091B9
:1020F0008F0F041710F40C9486100091210A003001
:1021000011F00C94861086E08093890F0091890F5E
:10211000033081E009F080E08F930091890F053052
:1021200081E009F080E09F91892B882311F40C94C1
:10213000A0108AE0A6EDBEE00E94CA290C94A81067
:10214000A6EDBEE0E2EDF5E60E94F8310E949E3178
:102150004091480A0091B10F041780E010F009F097
:1021600081E08F9340914A0A0091B10F041781E0FA
:1021700008F080E09F918923882311F40C94D610F5
:102180000091890F033081E009F080E08F93009186
:10219000890F043081E009F080E09F91892B88232A
:1021A00011F40C94D61085E08093890F4091470A72
:1021B0000091B10F041781E010F009F080E08F93D7
:1021C0004091490A0091B10F041781E008F480E0C2
:1021D0009F91892B882311F40C940F110091210AEF
:1021E000003011F00C94F91070916F0072607093D0
:1021F0006F000091890F023081E009F080E08F9339
:102200000091890F053081E009F080E09F91892BD2
:10221000882311F40C940F1183E08093890F0C94A0
:1022200094110091890F023011F40C941A1180E07E
:1022300080938F0F4091900F00918F0F041710F42F
:102240000C942B110091210A003011F00C942B11E9
:1022500086E08093890F0091890F033081E009F0B7
:1022600080E08F930091890F053081E009F080E0D4
:102270009F91892B882311F40C9445118AE0A6EDD7
:10228000BEE00E94CA290C944D11A6EDBEE0E2ED1D
:10229000F5E60E94F8310E949E3140914A0A009171
:1022A000B10F041710F00C946B110091890F0330DB
:1022B00081E009F080E08F930091890F043081E084
:1022C00009F080E09F91892B882311F40C946B1105
:1022D00085E08093890F4091490A0091B10F04175E
:1022E00010F40C9494110091210A003011F00C9418
:1022F0007E1170916F00726070936F000091890F72
:10230000023081E009F080E08F930091890F053061
:1023100081E009F080E09F91892B882311F40C94CF
:10232000941183E08093890F0091890F063011F496
:102330000C94E5118AE00E94E829082F0F3F11F064
:102340000C94E3110091890F023081E009F080E0E4
:102350008F930091890F043081E009F080E09F9114
:10236000892B882311F40C94C411A5ECBEE0E2ED96
:10237000F5E60E94F8310E949E318AE0A5ECBEE0AD
:102380000E94D2290C94E3110091890F013081E061
:1023900009F080E08F930091890F053081E009F00A
:1023A00080E09F91892B882311F40C94DA1182E04C
:1023B0008093890F0091890F033011F00C94E31181
:1023C00084E08093890F0C94F5118AE00E94E8293B
:1023D000082F0F3F11F00C94F51170916F007D7F65
:1023E00070936F0081E08093890F4091890F009175
:1023F0008A0F041711F40C9408120E9474198AE0D1
:102400000E94DF290E948F198091890F80938A0F83
:1024100008950091B00F003011F00C94101208953F
:1024200000911B0A013011F40C94101600912E0A31
:10243000003011F00C94B9124091430A0091B00F92
:10244000041781E010F009F080E08F930091B60F3F
:102450000F3F81E009F080E09F918923882311F4E8
:102460000C94711280E08093B60F00911B0A00302B
:1024700081E009F080E08F9300911B0A033081E036
:1024800009F080E09F91892B8F930091210A013000
:1024900081E009F080E09F918923882311F40C9456
:1024A0006412AFE6B0E00C9101FB16F40C945F12DD
:1024B00070916F00726070936F000C94621286E0EE
:1024C0008093890F0C947112A9E6BAE0E2E9F7E66D
:1024D0000E94F8310E946B318BE00E94DF290E943C
:1024E000171B4091450A0091B00F041781E008F4D2
:1024F00080E08F930091B60F0F3F81E009F080E0FC
:102500009F918923882311F40C94961280E0809384
:10251000B60FA9E6BAE0EEE9F7E60E94F8310E94AC
:102520006B318BE00E94DF290E94171B00913A0A51
:10253000003011F40C94B9124091440A0091B00F8C
:10254000041781E008F480E08F934091460A0091DF
:10255000B00F041781E010F009F080E09F9189230B
:10256000882311F40C94B912709171007D7F7093DF
:10257000710000912E0A013011F00C94FA130091B1
:10258000B60F0F3F11F00C94E2124091430A0091F4
:10259000B00F041718F011F00C94D41281E080935E
:1025A0007A0F81E080937B0F4091450A0091B00F34
:1025B000041710F40C94E21281E080937A0F82E009
:1025C00080937B0F00913F0A0C3010F40C94DF13C2
:1025D0004091440A0091B00F041710F40C94F912C2
:1025E00000917B0F013011F00C94F9128FEF809362
:1025F0007D0F4091460A0091B00F041718F011F0BA
:102600000C940B1300917B0F023011F00C940B1300
:102610008FEF80937D0F00913F0A0A3710F40C94DE
:1026200014138FEF80937D0F00917D0F0F3F11F0FA
:102630000C94DD1300913F0A0A3710F40C94321306
:1026400000917B0F013011F00C94291383E08093EB
:102650007B0F00917B0F023011F00C94321384E059
:1026600080937B0F00911B0A003081E009F080E02D
:102670008F9300911B0A033081E009F080E09F9165
:10268000892B8F930091210A013081E009F080E0CD
:102690009F9189238F9300917B0F013081E009F096
:1026A00080E09F918923882311F40C946A13AFE68C
:1026B000B0E00C9101FB16F40C94651370916F005F
:1026C000726070936F000C94681386E08093890F9A
:1026D0000C94CA1300917B0F013011F00C947A1303
:1026E000A9E6BAE0E2E9F7E60E94F8310E946B3110
:1026F0000C94A213023011F00C948813A9E6BAE0EE
:10270000EEE9F7E60E94F8310E946B310C94A213B7
:10271000033011F00C949613A9E6BAE0EAEAF7E662
:102720000E94F8310E946B310C94A213043011F016
:102730000C94A213A9E6BAE0E6EBF7E60E94F831A2
:102740000E946B3100913A0A013081E009F080E08B
:102750008F9340917B0F00917C0F041781E009F06B
:1027600080E09F918923882311F40C94BF1380E0AB
:1027700080937B0F709171007D7F70937100009149
:102780007B0F003011F40C94CA138BE00E94DF29F8
:102790000E94171B80917B0F80937C0F80E08093B9
:1027A0007B0F80E080937A0F80E080933F0A80E087
:1027B00080937D0F80E08093B60F0C94FA134091C4
:1027C000440A0091B00F041781E008F480E08F9371
:1027D0004091460A0091B00F041781E010F009F013
:1027E00080E09F918923882311F40C94FA1380E0F0
:1027F00080937A0F00912E0A023011F00C9470151C
:102800004091430A0091B00F041781E010F009F0E5
:1028100080E08F934091450A0091B00F041781E04A
:1028200008F480E09F91892B882311F40C942914DB
:102830000091B60F0F3F11F00C94271480E08093A5
:10284000B60F81E080937A0F80E08093800F0C9424
:10285000501400913F0A0C3081E008F480E08F931F
:1028600000913F0A0A3781E008F080E09F918923B8
:10287000882311F40C94501400917B0F083010F051
:102880000C944714ABE7BFE08C918F5F8C9381E091
:1028900080937F0F80E080937A0F80E080933F0ADF
:1028A00000913F0A0A3710F40C94611580E0809380
:1028B0007A0F80E080933F0A00917B0F003011F087
:1028C0000C94661480917C0F80937B0F00911B0AFF
:1028D000003081E009F080E08F9300911B0A033003
:1028E00081E009F080E09F91892B8F930091210A6C
:1028F000013081E009F080E09F9189238F9300915E
:102900007B0F013081E009F080E09F9189238823CB
:1029100011F40C949E14AFE6B0E00C9101FB16F498
:102920000C94991470916F00726070936F000C9406
:102930009C1486E08093890F0C945A1500917F0FA8
:10294000003011F40C945A1500917B0F013011F0F6
:102950000C94B414A9E6BAE0E2E9F7E60E94F83173
:102960000E946B310C941415023011F00C94C214B7
:10297000A9E6BAE0EEE9F7E60E94F8310E946B3171
:102980000C941415033011F00C94D014A9E6BAE09D
:10299000EAEAF7E60E94F8310E946B310C941415B4
:1029A000043011F00C94DE14A9E6BAE0E6EBF7E689
:1029B0000E94F8310E946B310C941415053011F00F
:1029C0000C94EC14A9E6BAE0E2ECF7E60E94F831C8
:1029D0000E946B310C941415063011F00C94FA140B
:1029E000A9E6BAE0EEECF7E60E94F8310E946B31FE
:1029F0000C941415073011F00C940815A9E6BAE0F0
:102A0000EAEDF7E60E94F8310E946B310C94141540
:102A1000083011F00C941415A9E6BAE0E6EEF7E6DA
:102A20000E94F8310E946B3100913A0A013081E036
:102A300009F080E08F9300917E0F003081E009F46F
:102A400080E09F9189238F9340917C0F00917B0FB1
:102A5000041781E009F080E09F918923882311F415
:102A60000C943F1580E080937E0F80E080937B0F75
:102A7000709171007D7F709371000C945A150091D4
:102A80007B0F003081E009F480E08F9300917E0F8E
:102A9000003081E009F080E09F91892B882311F4B8
:102AA0000C945A158BE00E94DF290E94171B81E0CD
:102AB00080937E0F80917B0F80937C0F80E08093CA
:102AC0007B0F00917B0F003011F40C947015009176
:102AD000800F033010F40C94701580E080937B0F0E
:102AE000A9E6BAE0E2E9F7E60E94F8310E94C532B1
:102AF00011F00C948415ABE3BAE08C9187FBAAE348
:102B0000BAE0882780F98C93A9E6BAE0EEE9F7E607
:102B10000E94F8310E94C53211F00C949815ABE375
:102B2000BAE08C9186FBAAE3BAE0882780F98C93FF
:102B3000A9E6BAE0EAEAF7E60E94F8310E94C53257
:102B400011F00C94AC15ABE3BAE08C9185FBAAE3D1
:102B5000BAE0882780F98C93A9E6BAE0E6EBF7E6BD
:102B60000E94F8310E94C53211F00C94C015ABE3FD
:102B7000BAE08C9184FBAAE3BAE0882780F98C93B1
:102B8000A9E6BAE0E2ECF7E60E94F8310E94C5320D
:102B900011F00C94D415ABE3BAE08C9183FBAAE35B
:102BA000BAE0882780F98C93A9E6BAE0EEECF7E664
:102BB0000E94F8310E94C53211F00C94E815ABE385
:102BC000BAE08C9182FBAAE3BAE0882780F98C9363
:102BD000A9E6BAE0EAEDF7E60E94F8310E94C532B4
:102BE00011F00C94FC15ABE3BAE08C9181FBAAE3E5
:102BF000BAE0882780F98C93A9E6BAE0E6EEF7E61A
:102C00000E94F8310E94C53211F00C941016ABE30B
:102C1000BAE08C9180FBAAE3BAE0882780F98C9314
:102C200008950091B10F003011F00C94181608951A
:102C300000912D0A003011F00C948C164091470A37
:102C40000091B10F041781E010F009F080E08F933C
:102C50000091B70F0F3F81E009F080E09F91892339
:102C6000882311F40C94441680E08093B70FA8E7F2
:102C7000BAE0E2EFF7E60E94F8310E946B318AE099
:102C80000E94DF290E94681A4091490A0091B10F01
:102C9000041781E008F480E08F930091B70F0F3F95
:102CA00081E009F080E09F918923882311F40C943E
:102CB000691680E08093B70FA8E7BAE0EEEFF7E679
:102CC0000E94F8310E946B318AE00E94DF290E9445
:102CD000681A0091390A003011F40C948C16409156
:102CE000480A0091B10F041781E008F480E08F9347
:102CF00040914A0A0091B10F041781E010F009F0E9
:102D000080E09F918923882311F40C948C16709194
:102D10006F007D7F70936F0000912D0A013011F0DC
:102D20000C9495170091B70F0F3F11F00C94B51646
:102D30004091470A0091B10F041718F011F00C945C
:102D4000A71681E08093810F81E08093820F4091EC
:102D5000490A0091B10F041710F40C94B51681E0E4
:102D60008093810F82E08093820F0091400A0C30A3
:102D700010F40C947A174091480A0091B10F04178F
:102D800010F40C94CC160091820F013011F00C94C9
:102D9000CC168FEF8093840F40914A0A0091B10FB7
:102DA000041718F011F00C94DE160091820F023017
:102DB00011F00C94DE168FEF8093840F0091400A7F
:102DC0000A3710F40C94E7168FEF8093840F00916C
:102DD000840F0F3F11F00C9478170091400A0A37C6
:102DE00010F40C9405170091820F013011F00C942F
:102DF000FC1683E08093820F0091820F023011F065
:102E00000C94051784E08093820F0091820F0130AB
:102E100011F00C941517A8E7BAE0E2EFF7E60E946C
:102E2000F8310E946B310C943D17023011F00C9474
:102E30002317A8E7BAE0EEEFF7E60E94F8310E9408
:102E40006B310C943D17033011F00C943117A8E747
:102E5000BAE0EAE0F8E60E94F8310E946B310C9487
:102E60003D17043011F00C943D17A8E7BAE0E6E1F5
:102E7000F8E60E94F8310E946B310091390A013066
:102E800081E009F080E08F934091820F0091830FE1
:102E9000041781E009F080E09F918923882311F4D1
:102EA0000C945A1780E08093820F70916F007D7FA1
:102EB00070936F000091820F003011F40C9465172D
:102EC0008AE00E94DF290E94681A8091820F809315
:102ED000830F80E08093820F80E08093810F80E0F9
:102EE0008093400A80E08093840F80E08093B70F46
:102EF0000C9495174091480A0091B10F041781E096
:102F000008F480E08F9340914A0A0091B10F0417B2
:102F100081E010F009F080E09F918923882311F46B
:102F20000C94951780E08093810F00912D0A023058
:102F300011F00C94D3184091470A0091B10F041777
:102F400081E010F009F080E08F934091490A0091F0
:102F5000B10F041781E008F480E09F91892B88234A
:102F600011F40C94C4170091B70F0F3F11F00C949B
:102F7000C21780E08093B70F81E08093810F80E0DB
:102F80008093870F0C94EB170091400A0C3081E07E
:102F900008F480E08F930091400A0A3781E008F03E
:102FA00080E09F918923882311F40C94EB17009102
:102FB000820F083010F00C94E217A2E8BFE08C9169
:102FC0008F5F8C9381E08093860F80E08093810FE8
:102FD00080E08093400A0091400A0A3710F40C9474
:102FE000C41880E08093810F80E08093400A0091B4
:102FF000860F003011F40C94C4180091820F003039
:1030000011F00C9407188091830F8093820F009128
:10301000820F013011F00C941718A8E7BAE0E2EF24
:10302000F7E60E94F8310E946B310C947718023059
:1030300011F00C942518A8E7BAE0EEEFF7E60E942D
:10304000F8310E946B310C947718033011F00C9416
:103050003318A8E7BAE0EAE0F8E60E94F8310E94E7
:103060006B310C947718043011F00C944118A8E7D8
:10307000BAE0E6E1F8E60E94F8310E946B310C9468
:103080007718053011F00C944F18A8E7BAE0E2E287
:10309000F8E60E94F8310E946B310C9477180630E4
:1030A00011F00C945D18A8E7BAE0EEE2F8E60E9491
:1030B000F8310E946B310C947718073011F00C94A2
:1030C0006B18A8E7BAE0EAE3F8E60E94F8310E943C
:1030D0006B310C947718083011F00C947718A8E72E
:1030E000BAE0E6E4F8E60E94F8310E946B31009104
:1030F000390A013081E009F080E08F930091850F5B
:10310000003081E009F480E09F9189238F93409102
:10311000830F0091820F041781E009F080E09F91F6
:103120008923882311F40C94A21880E08093850FE2
:1031300080E08093820F70916F007D7F70936F00AD
:103140000C94BD180091820F003081E009F480E0FA
:103150008F930091850F003081E009F080E09F910E
:10316000892B882311F40C94BD188AE00E94DF2972
:103170000E94681A81E08093850F8091820F80936E
:10318000830F80E08093820F0091820F003011F452
:103190000C94D3180091870F033010F40C94D318BB
:1031A00080E08093820FA8E7BAE0E2EFF7E60E94A2
:1031B000F8310E94C53211F00C94E718ACE3BAE084
:1031C0008C9187FBA9E3BAE0882780F98C93A8E764
:1031D000BAE0EEEFF7E60E94F8310E94C53211F036
:1031E0000C94FB18ACE3BAE08C9186FBA9E3BAE03F
:1031F000882780F98C93A8E7BAE0EAE0F8E60E9415
:10320000F8310E94C53211F00C940F19ACE3BAE00A
:103210008C9185FBA9E3BAE0882780F98C93A8E715
:10322000BAE0E6E1F8E60E94F8310E94C53211F0FA
:103230000C942319ACE3BAE08C9184FBA9E3BAE0C7
:10324000882780F98C93A8E7BAE0E2E2F8E60E94CA
:10325000F8310E94C53211F00C943719ACE3BAE092
:103260008C9183FBA9E3BAE0882780F98C93A8E7C7
:10327000BAE0EEE2F8E60E94F8310E94C53211F0A1
:103280000C944B19ACE3BAE08C9182FBA9E3BAE051
:10329000882780F98C93A8E7BAE0EAE3F8E60E9471
:1032A000F8310E94C53211F00C945F19ACE3BAE01A
:1032B0008C9181FBA9E3BAE0882780F98C93A8E779
:1032C000BAE0E6E4F8E60E94F8310E94C53211F057
:1032D0000C947319ACE3BAE08C9180FBA9E3BAE0DB
:1032E000882780F98C930895AAE5BAE0E2E5F8E62C
:1032F0000E94F8310E946B31E9E8FFE0AAE5BAE0EC
:103300000E94B4250E942B32AAE5BAE00E94B4259F
:10331000EAE5F8E60E94F8310E946B3108958AE0F0
:10332000AAE5BAE00E94AE298AE0ADEABEE00E94BA
:10333000C42907E110E020E030E068948AE0A3EAC5
:10334000BEE00E94182A09E110E020E030E0689415
:103350008AE0A7EABEE00E94162A09E210E020E017
:1033600030E068948AE0A4E9BEE00E94142A00E0FC
:1033700014E224EF30E0A7EABEE04D915C916627AD
:1033800077270E94D725A5ECBEE04D935D936D9302
:103390007D93A5ECBEE08D919C91909389008093E4
:1033A0008800A8E8B0E08D919C91A6E7BFE08D93DE
:1033B0009C93A2EDBEE0E2EDF5E60E94F8310E949A
:1033C0009E3100911B0A033010F40C94201A0091D6
:1033D000890F033081E009F080E08F930091890F1D
:1033E000053081E009F080E09F91892B882311F45A
:1033F0000C94201A4DE250E060E070E0A6EDBEE0D3
:103400000D911D912D913C910E9408321CF011F0FC
:103410000C940C1A0C94201AADEABEE00D911D918B
:103420002D913C91A6EDBEE04D915D916D917C9109
:103430000E940332A2EDBEE00D931D932D933D93A8
:10344000A2EDBEE00D911D912D913C91A5ECBEE049
:103450000D931D932D933C938AE0A5ECBEE00E9452
:10346000D229A4E9BEE00D911D912D913C9140E03F
:1034700054E060E070E00E94D725A9EBBEE04D93D8
:103480005D936D937D93A9EBBEE00D911D912D9100
:103490003C9140E054E060E070E00E944831A9EBCC
:1034A000BEE00D931D932D933D93A9EBBEE00D91CE
:1034B0001D912D913C914CE250E060E070E00E9443
:1034C000FE31A9EBBEE00D931D932D933D9308951E
:1034D000A8E7BAE0E0E1F0E00E94322A40E050E0E4
:1034E00060E070E00E9408321CF011F00C947A1A2F
:1034F0000C94111B8AE0A8E7BAE00E94AE298AE08A
:10350000A5EBBEE00E94C42907E110E020E030E016
:1035100068948AE0A3EABEE00E94182A09E110E05C
:1035200020E030E068948AE0A7EABEE00E94162A14
:1035300009E210E020E030E068948AE0A4E9BEE00F
:103540000E94142A00E014E224EF30E0A7EABEE073
:103550004D915C91662777270E94D725A5ECBEE0A8
:103560004D935D936D937D93A5ECBEE08D919C9101
:103570009093890080938800A5ECBEE0E2EDF5E62B
:103580000E94F8310E949E318AE0A5ECBEE00E94C4
:10359000D229A4E9BEE00D911D912D913C9140E00E
:1035A00054E060E070E00E94D725A1ECBEE04D93AE
:1035B0005D936D937D93A1ECBEE00D911D912D91D6
:1035C0003C9140E054E060E070E00E944831A1ECA2
:1035D000BEE00D931D932D933D93A1ECBEE00D91A4
:1035E0001D912D913C914CE250E060E070E00E9412
:1035F000FE31A1ECBEE00D931D932D933D930E94EF
:10360000010C0E94600C80E080939E0EA0E9BAE25B
:103610000E94A63170916F00726070936F000C94DD
:10362000161B70916F007D7F70936F000895A9E65F
:10363000BAE0E0E1F0E00E94322A40E050E060E0D1
:1036400070E00E9408321CF011F00C94291B0C94BD
:10365000C01B8BE0A9E6BAE00E94AE298BE0A1EB8B
:10366000BEE00E94C42907E110E020E030E0689449
:103670008BE0A4EABEE00E94182A09E110E020E0F5
:1036800030E068948BE0A9EABEE00E94162A09E2C5
:1036900010E020E030E068948BE0A8E9BEE00E94F2
:1036A000142A00E014E224EF30E0A9EABEE04D91D4
:1036B0005C91662777270E94D725A9ECBEE04D9341
:1036C0005D936D937D93A9ECBEE08D919C91909359
:1036D000990080939800A9ECBEE0E2EDF5E60E9427
:1036E000F8310E949E318BE0A9ECBEE00E94D22905
:1036F000A8E9BEE00D911D912D913C9140E054E070
:1037000060E070E00E94D725ADEBBEE04D935D9385
:103710006D937D93ADEBBEE00D911D912D913C918C
:1037200040E054E060E070E00E944831ADEBBEE064
:103730000D931D932D933D93ADEBBEE00D911D9127
:103740002D913C914CE250E060E070E00E94FE312F
:10375000ADEBBEE00D931D932D933D930E94BF0CE6
:103760000E94080D80E08093A20EA2E9BAE20E94B6
:10377000A631709171007260709371000C94C51B3A
:10378000709171007D7F70937100089580E0809347
:103790009F0EABEABEE00E94A63181E08093890FC4
:1037A0000091890F063018F011F00C94A41CA7EAC0
:1037B000BEE00E94A63180E08093A30EA5EABEE0A1
:1037C0000E94A631ADEABEE00E94A831A7E8BAE0A7
:1037D0000E94A6310E947419AAE5BAE0E0E1F0E087
:1037E0000E94322A40E050E060E070E00E9408321F
:1037F00011F00C94001C81E080939F0E0C94A41C8B
:103800008AE0AAE5BAE00E94AE2900919F0E00303E
:1038100011F00C949C1C09E010E020E030E068946A
:1038200044E08AE0A7E8BAE00E941A2A88278C932D
:10383000A7E8BAE0E0E6F8E60E94F8310E94C53257
:1038400011F40C942B1C82E080939F0E8AE00E945E
:10385000DF290C94A41C07E110E020E030E068941C
:103860008AE0A3EABEE00E94182A0091A30E03306A
:1038700010F40C94431C83E080939F0E8AE00E9416
:10388000DF290C94A41C09E110E020E030E06894EA
:103890008AE0A7EABEE00E94162AA7EABEE00D91E0
:1038A0001C9100345FE1150781E009F480E08F93FB
:1038B000A7EABEE00D911C9101315BE2150781E0A2
:1038C00009F480E09F9189238F93A7EABEE00D91D0
:1038D0001C91023256E5150781E009F480E09F91C2
:1038E0008923882311F40C947D1C84E080939F0E1F
:1038F0008AE00E94DF290C94A41C03E210E020E07F
:1039000030E068948AE0A5EABEE00E94162AA5EAA3
:10391000BEE00D911C91083050E0150711F40C9495
:10392000991C85E080939F0E8AE00E94DF290C9409
:10393000A41C8AE00E94DF29A9E8BFE08C918F5F78
:103940008C9310F40C94D01B00919F0E003011F456
:103950000C94E91C5D980091890F42E0049FA8EE49
:10396000BEE00C92E2E1F6E60E94F8310E94C32527
:10397000E9E8FFE0A0E8BFE30E942B320E94BB25EC
:103980000E94CA2580E289B98AEF90E00E948526CC
:103990008091E80E81508093E80E0091E80E00308F
:1039A00011F00C94DF1C5D980091890F42E0049F98
:1039B000A8EEBEE00C928AEC98E00E948526009169
:1039C000BA0F003411F00C94E71C0C94F21C0C9408
:1039D000C21CEEE0F6E60E94F8310E94C3250E9468
:1039E000CA2508959FB7F8948091600088618093FC
:1039F0006000877E809360009FBFE898E99870918F
:103A00006E007E7F70936E0070916F007D7F70936B
:103A10006F0070916F007B7F70936F0070917100E9
:103A20007D7F70937100709171007B7F7093710046
:103A3000882785BD80918100887F809381008827B9
:103A40008093B10080919100887F809391001798B6
:103A50005D98529A5A9A53980E94301FA1E9BFE08C
:103A60000E94A6310E947326A5EEBEE08C930091C1
:103A7000E50E0D3011F40C94491DA5EEBEE08C91BD
:103A8000A1E9BFE00E94B4258D9388278C930C9404
:103A90002E1FA1E9BFE0E6E6F8E60E94F8310E9499
:103AA000C53211F00C94561D0E94301FA1E9BFE0F1
:103AB000E8E6F8E60E94F8310E94C53211F00C9455
:103AC000691DEEE6F8E60E94F8310E9457260E9432
:103AD0005E26A1E9BFE0ECE7F8E60E94F8310E941B
:103AE000C53211F00C94C21D80E08093EB0E81E092
:103AF0008093E60E0091E60E0F3518F011F00C944D
:103B0000A21DA6EEBEE0EC91FF27AFEEBEE091E075
:103B10000E94BE320091EB0E4091EF0E040FABEE0F
:103B2000BEE00C93EFEEFEE0A0E8BFE30E9471322E
:103B30000E946226A6EEBEE08C918F5F8C9310F4FB
:103B40000C947A1DE6E6F0E0A0E8BFE30E94713233
:103B50000E9462260091EB0E40916600040FABEECE
:103B6000BEE00C93EBEEFEE0A0E8BFE30E947132F2
:103B70000E946226E2E8F8E60E94F8310E94572689
:103B80000E945E26A1E9BFE0EAE8F8E60E94F8316B
:103B90000E94C53211F00C94151FE0E9F8E60E946E
:103BA000F8310E9457260E945E2680E08093E60E40
:103BB00080E080939C0F80E08093EB0EACEEBEE043
:103BC0000E94A6310E947326A5EEBEE08C93009160
:103BD000E50E0D3011F00C94EF1D0C941F1EA5EE98
:103BE000BEE08C91ACEEBEE00E94B4258D93882798
:103BF0008C93A6EEBEE08C918F5F8C930091E60EC5
:103C0000023011F00C941D1EACE9BFE08C918F5F67
:103C10008C93ACEEBEE00E948A32ACE9BFE0AD907E
:103C2000BB24AFEEBEE0AA0DBB1D0C93ACEEBEE014
:103C30000E94A63180E08093E60E0C94E21D009174
:103C40009C0F41E0041BA7EEBEE00C938091E70EB1
:103C5000E0EFFEE00E94D932ABEEBEE00C93ACE99F
:103C6000BFE0AD90BB24AFEEBEE0AA0DBB1D4C91F2
:103C70000091EB0E041711F00C940D1F0091F00E43
:103C8000023011F00C94031F8091F10E8093E90E25
:103C90000091F10E4091F20E040FAAEEBEE00C93DB
:103CA0008091EA0E81508093EA0E84E08093E70EC3
:103CB0008091E90E8093E60E4091EA0E0091E60EA7
:103CC000041718F011F00C94DC1E0091F20E0F3561
:103CD00011F00C947D1EA6EEBEE0EC91FF27A7EE3E
:103CE000BEE0AD90BB24AFEEBEE0AA0DBB1D91E0DF
:103CF0007BE70E94AD320C94CF1E0091E60E0D3191
:103D000081E009F480E08F930091E60E0E3181E0AE
:103D100009F480E09F9189238F930091E60E0F3183
:103D200081E009F480E09F918923882311F40C94A9
:103D3000CF1E0091E60E0C3281E009F480E08F93F3
:103D40000091E60E0D3281E009F480E09F91892315
:103D5000882311F40C94CF1E0091E60E0E3281E000
:103D600009F480E08F930091E60E0F3281E009F4B0
:103D700080E09F918923882311F40C94CF1EA6EE36
:103D8000BEE0EC91FF27A7EEBEE0AD90BB24AFEE06
:103D9000BEE0AA0DBB1D91E07BE70E94AD32A7EE0D
:103DA000BEE08C918F5F8C93A6EEBEE08C918F5F0E
:103DB0008C9310F40C945C1EE4E9F8E60E94F83150
:103DC0000E9457260E945E26ABE4BAE0ECECF6E6D1
:103DD0000E94F8310E946B31ABE4BAE0E0E1F0E020
:103DE0000E94322A40E050E060E070E00E94083219
:103DF00011F40C94011FABE4BAE00E942F2D0E9435
:103E0000832E0C940B1FECE9F8E60E94F8310E9417
:103E100057260E945E260C94151FE4EAF8E60E94DD
:103E2000F8310E9457260E945E26A1E9BFE0ECEA25
:103E3000F8E60E94F8310E94C53211F00C942A1F56
:103E4000E0EBF8E60E94F8310E9457260E945E26B9
:103E50000C944C1FA1E9BFE00E94A6310C94321DC6
:103E60004C9B0C943D1FA1E9BFE0E6EBF8E60E94F5
:103E7000F8310E946B310C94451FA1E9BFE0E2ECE0
:103E8000F8E60E94F8310E946B31A1E9BFE00E9480
:103E900064260E945E260895A89574B7777F74BF44
:103EA00088E190E0809360009093600080916000D2
:103EB00088608093600000000C945B1F089500915F
:103EC000BB0F003011F00C94851FAFE6B0E00C91F1
:103ED00001FB16F00C94741F70916F007D7F70933E
:103EE0006F0081E08093BB0FA1E7B0E00C9101FB74
:103EF00016F00C94851F709171007D7F7093710096
:103F0000ABEBBFE08C918E5F8C93479A82E08093FD
:103F1000B1007CE27093B3007CE27093B40082E362
:103F200090E00E94852681E08093B10082E390E0DA
:103F30000E94852608950091BB0F003011F00C946B
:103F4000C11FAFE6B0E00C9101FB16F00C94B01F5E
:103F500070916F007D7F70936F0081E08093BB0F45
:103F6000A1E7B0E00C9101FB16F00C94C11F709119
:103F700071007D7F70937100ABEBBFE08C918E5F21
:103F80008C93479A82E08093B1007CE27093B300F7
:103F90007CE27093B40084E690E00E94852681E084
:103FA0008093B10084E690E00E94852608950091F8
:103FB0007C00007E036000937C000E947131AEEDB6
:103FC000BEE08D939D9388278D938C93AEEDBEE0DC
:103FD0000D911D912D913C9149E150E060E070E020
:103FE0000E944831AEEDBEE00D931D932D933D939D
:103FF000AEEDBEE00D911D912D913C9148E250E057
:1040000060E070E00E94D725AEEDBEE04D935D9379
:104010006D937D93ACEDBEE00D911C91003050E0AE
:10402000150711F40C942D20AEEDBEE00D911D91FD
:104030002D913C91ACEDBEE04D915D9157FB1EF48E
:104040006FEF7FEF02C0662777270E94FE31AEED4B
:10405000BEE00D931D932D933D93AEEDBEE08D918B
:104060009C91AAEDBEE08D939C930091220A0030B2
:1040700011F40C946E20A4E2BAE04D915C91AAED8B
:10408000BEE00D911C910417150710F00C944B2005
:1040900081E08093E20EA6E2BAE04D915C91AAED38
:1040A000BEE00D911C910417150718F011F00C9447
:1040B0005B200C945E2080E08093E20E0091E20E83
:1040C000013011F00C946A2080E289B90E949B1F94
:1040D0000C946E205D9880E08093E20E4C9B0C94D3
:1040E0008220AAEDBEE00D911C91083552E0150723
:1040F00018F011F00C947E200C9480200E949220E5
:104100000C949120AAEDBEE00D911C910A3852E06A
:10411000150718F011F00C948F200C9491200E9438
:1041200092200895789417985D9881E08093E30E2B
:10413000EDE1F0E0A4EEBEE091E00E94BE3200911D
:10414000E40E0F3F81E009F080E08F930091E40ED0
:104150000A3181E009F080E09F91892B882311F4D6
:104160000C94B52080E08093E40EA4EEBEE08C9128
:104170008F5F8C93EDE1F0E0A4EEBEE091E07BE791
:104180000E94AD32EEE1F0E0AAEDBEE092E07BE706
:104190000E94AD3280E880B980E289B90E949B1FFD
:1041A0000091BA0F003411F00C94D8200C94F21C3A
:1041B0000C94CA2008955D9A8AEF90E00E948526AB
:1041C0005D980895F894FFCF0F931F938F939F935B
:1041D000AF93BF930FB70F938091902A9091912A3C
:1041E00001968093902A9093912A00919E0E00232D
:1041F000F9F4A0E9BAE20D911D91AFE8BAE0A00F81
:10420000B11F0C910093B3000091A30E023009F48A
:104210000196A0918C0AB0918D0A8A179B0728F10C
:104220008827992780939C0E01E000939E0E1DC065
:10423000A0E9BAE20D911D91AFE8B2E1A00FB11F64
:104240000C910093B3000091A30E023009F4019683
:10425000A0918E0AB0918F0A8A179B0730F08827A9
:10426000992780939D0E80939E0E8093902A909321
:10427000912A0F910FBFBF91AF919F918F911F9185
:104280000F9118954F935F938F939F93AF93BF9325
:104290004FB74F938091922A9091932A01968093E1
:1042A000922A9093932A4091A20E4423F9F4A2E912
:1042B000BAE24D915D91AFE8BAE1A40FB51F4C9100
:1042C0004093B4004091A40E423009F40196A091AD
:1042D000900EB091910E8A179B0728F18827992795
:1042E0008093A00E41E04093A20E1DC0A2E9BAE265
:1042F0004D915D91AFE8B2E2A40FB51F4C91409390
:10430000B4004091A40E423009F40196A091920E9F
:10431000B091930E8A179B0730F0882799278093D6
:10432000A10E8093A20E8093922A9093932A4F918C
:104330004FBFBF91AF919F918F915F914F91189512
:104340000F921F922F923F924F925F927F92AF9265
:10435000BF920F931F932F933F934F935F936F934E
:104360007F938F939F93AF93BF93CF93DF93EF93FD
:10437000FF938FB78F938BB78F9388278BBFAEEA4E
:10438000BFE086B58C93A9E6B0E00C9100FB16F077
:104390000C94D8218091AE0F8093A40F80E080937D
:1043A000A20F709169007E7F709369000C94772250
:1043B0000091A20F013018F011F00C940622A5EA2A
:1043C000BFE086B58C934091A50F0091A40F041710
:1043D00010F40C94FC2100E04091A40F041BA4EA0B
:1043E000BFE00C930091A40F4091A50F040FA8EB20
:1043F000BFE00C930C9404220091A50F4091A40FF0
:10440000041BA8EBBFE00C930C9408220E94D62456
:10441000A8EABFE08C918F5F8C930091B40F0130BC
:1044200011F00C9436220091B80F0D3518F011F0F0
:104430000C942A220EE54091B80F041BA8EBBFE0B4
:104440000C930EE54091B80F040FA8EBBFE00C935E
:104450000C943622A8EBBFE08C918E558C930EE520
:104460004091B80F041BA8EBBFE00C930091B80F6C
:10447000003381E008F480E08F930091B80F0C388E
:1044800081E010F009F080E09F918923882311F4E6
:104490000C946B228091B80F8093B20F4091A90FBA
:1044A0000091B80F041781E008F480E08F934091E9
:1044B000AA0F0091B80F041781E010F009F080E016
:1044C0009F918923882311F40C9469228FEF8093A4
:1044D000B60F0C946D220E94D6248091B80F809361
:1044E000B00F70916900716070936900E09A8F91CC
:1044F0008BBF8F918FBFFF91EF91DF91CF91BF91D4
:10450000AF919F918F917F916F915F914F913F916B
:104510002F911F910F91BF90AF907F905F904F9020
:104520003F902F901F900F9018950F921F922F92EF
:104530003F924F925F927F92AF92BF920F931F93E1
:104540002F933F934F935F936F937F938F939F939B
:10455000AF93BF93CF93DF93EF93FF938FB78F9377
:104560008BB78F9388278BBFAFEABFE086B58C935C
:10457000A9E6B0E00C9102FB16F00C94CD228091DC
:10458000AF0F8093A60F80E08093A30F7091690016
:104590007B7F709369000C941C240091A30F013061
:1045A00018F011F00C94FB22A7EABFE086B58C93BB
:1045B0004091A70F0091A60F041710F40C94F1225C
:1045C00000E04091A60F041BA6EABFE00C93009107
:1045D000A60F4091A70F040FA9EBBFE00C930C941A
:1045E000F9220091A70F4091A60F041BA9EBBFE091
:1045F0000C930C94FD220E94EA24A8EABFE08C915F
:104600008F5F8C93ACE9BFE08C918F5F8C930091AE
:104610009C0F063010F00C9418238091B90FACE970
:10462000BFE0AD90BB24ACE9BFE0AA0DBB1D8C93ED
:1046300000919D0F053081E009F080E08F9300919B
:104640009D0F063081E009F080E09F91892B8F93C8
:1046500000919D0F073081E009F080E09F91892B48
:10466000882311F40C94A72300919E0F023181E05E
:1046700009F080E08F9300919E0F033181E009F0F3
:1046800080E09F91892B8F9300919E0F043181E0F0
:1046900009F080E09F91892B882311F40C94A723C3
:1046A00000919F0F053081E009F080E08F93009129
:1046B0009F0F063081E009F080E09F91892B8F9356
:1046C00000919F0F073081E009F080E09F91892BD6
:1046D000882311F40C94A7230091A00F053081E0EA
:1046E00009F080E08F930091A00F063081E009F07F
:1046F00080E09F91892B8F930091A00F073081E07C
:1047000009F080E09F91892B882311F40C94A72352
:104710000091A10F0C3081E009F080E08F930091AF
:10472000A10F0D3081E009F080E09F91892B8F93DC
:104730000091A10F0E3081E009F080E09F91892B5C
:10474000882311F40C94A72380E48093BA0F00917E
:10475000B50F013011F00C94D0230091B90F0D3535
:1047600018F011F00C94C4230EE54091B90F041B0E
:10477000A9EBBFE00C930EE54091B90F040FA9EB34
:10478000BFE00C930C94D023A9EBBFE08C918E5525
:104790008C930EE54091B90F041BA9EBBFE00C937D
:1047A0000091B90F003381E008F480E08F9300910D
:1047B000B90F0C3881E010F009F080E09F91892357
:1047C000882311F40C9410248091B90F8093B30FB7
:1047D0004091AB0F0091B90F041781E008F480E01D
:1047E0008F934091AC0F0091B90F041781E010F046
:1047F00009F080E09F918923882311F40C9403240D
:104800008FEF8093B70F0091D00E0A3010F00C9408
:104810000E24A0EDBEE08C918F5F8C930C9412243B
:104820000E94EA248091B90F8093B10F70916900C2
:10483000746070936900E19A8F918BBF8F918FBFE5
:10484000FF91EF91DF91CF91BF91AF919F918F91A8
:104850007F916F915F914F913F912F911F910F9198
:10486000BF90AF907F905F904F903F902F901F90A0
:104870000F9018950F930FB70F930091A20F039508
:104880000093A20F0091A30F03950093A30F009133
:104890008C0F003029F000918D0F039500938D0F40
:1048A00000917A0F003039F000913F0A0F3F19F064
:1048B000039500933F0A0091810F003039F0009179
:1048C000400A0F3F19F003950093400A00918E0FA4
:1048D0000395043F80F000918F0F039500938F0F95
:1048E0000091800F03950093800F0091870F03952F
:1048F0000093870F002700938E0F0091A80F0430BC
:1049000080F000911D0A013060F00091E30E00304C
:1049100041F400270093A80F179902C0179A01C00D
:1049200017980091A20F0C3040F0009169000360CD
:10493000009369000CB301600CBB0091A30F0C3015
:1049400048F0009169000C6000936900E19A00272B
:1049500000939C0F0091A20F0E3380F00091200A6B
:10496000013021F400270093B80F08C00091200AFD
:10497000023021F40091B20F0093B80F0091A30F01
:104980000E3380F00091200A013021F400270093BB
:10499000B90F08C00091200A023021F40091B30F32
:1049A0000093B90F0F910FBF0F9118950091200A36
:1049B000013011F00C94DF2480E08093B80F009157
:1049C000200A023011F00C94E9248091B20F8093F8
:1049D000B80F08950091200A013011F00C94F324CF
:1049E00080E08093B90F0091200A023011F00C94FE
:1049F000FD248091B30F8093B90F089580E08093D8
:104A000003010E94E526AFEBBFE09C93A3E0B1E079
:104A10008C918F5F8C93469800910501003011F4C2
:104A20000C942425EEECF8E60E94F8310E94C32590
:104A3000E5E0F1E0A0E8BFE30E942B320E94BB2535
:104A40000E94CA250C942C25ECEDF8E60E94F83162
:104A50000E94C3250E94CA2581E00E94FE28A2E090
:104A6000B1E09C9300910201003011F40C944D25AB
:104A7000E8EEF8E60E94F8310E94C325E2E0F1E09A
:104A8000A0E8BFE30E942B320E94BB250E94CA25EA
:104A900080E0809300010C945825EEEFF8E60E9428
:104AA000F8310E94C3250E94CA2581E0809300014D
:104AB00000910201003081E009F080E08F930091C5
:104AC00003010A3081E008F480E09F91892B88235C
:104AD00011F40C940625469A0895ED91FC91E1504D
:104AE000F040FC93EE93089509D00E943E3100FC03
:104AF00010D0089503D01ED001F8F9CF0024E89417
:104B000057FF02C009D0689400F80BD010F80124B8
:104B1000089502D009D00895509540954F5F5F4F9A
:104B20000895E89417FF0895009510950F5F1F4FA3
:104B300068940895352F242FE894452B11F4689438
:104B40000895512F402F0027112780E1440F551F52
:104B5000001F111F021B130B416018F4020F131FDB
:104B60004E7F8A9599F708958F938D918823E9F761
:104B700011978F910895A0E8BFE38D91882311F0DC
:104B80000CD0FBCF08950E949031802D11F005D0FC
:104B9000FACF08958DE001D08AE00090C00005FEB4
:104BA000FCCF8093C600089500FC05D0089530D056
:104BB00005D001F8F9CF37D03FD00895842F952F35
:104BC000A62FB72FE894452B462B472B11F468945A
:104BD0000895402F512F622F732F0027112722276E
:104BE0003327F0E2440F551F661F771F001F111F68
:104BF000221F331F081B190B2A0B3B0B416028F4A3
:104C0000080F191F2A1F3B1F4E7FFA9559F7089569
:104C10000024E89477FF02C006D0689400F809D019
:104C200010F80124089512D04F5F5F4F6F4F7F4FF0
:104C30000895E89437FF08950095109520953095D4
:104C40000F5F1F4F2F4F3F4F689408954095509529
:104C50006095709508953197F1F70895279A2698F1
:104C60002E9A259A249A8CE58CBD0895089508956E
:104C7000689462F80895E89462F808958F939F937A
:104C80008BEC90E00197F1F79F918F9108958095BB
:104C90002AE090E0089410F45A9802C05A9A000052
:104CA000EDDFECDF969587952A95A9F708950E9488
:104CB0009031802D11F0EBDFFACF08958DE0E7DF22
:104CC0008AE0E5CFA0E8BFE38D91882311F0DFDF14
:104CD000FBCF08958F939F938BEC90E00197F1F7B2
:104CE0009F918F9108954B9B01C0FDCF29E04B9977
:104CF000FECFF0DFEFDFEEDF88944B9908942A9522
:104D000019F087959795F6CF0895EF93FF93EE27C7
:104D1000E82BE92B31F0E0EAFFE03197F1F701975A
:104D2000D1F7FF91EF910895689401C0E8948F93B3
:104D30009F9397E9000000009A95E1F7989480917D
:104D4000C20F9091C30F1EF4019708F4019680934F
:104D5000C20F9093C30F59F08091C00F9091C10F73
:104D6000019708F401968093C00F9093C10F9F9113
:104D70008F91089500E440E050E060E070E088C06A
:104D800008E44AEA51E0F9CF09E482C00AE480C0AD
:104D900000E540E052E0F1CF01E57AC008E578C0D7
:104DA0000AE7E9CF0DECE7CF09EEE5CF09EE40E0E9
:104DB00050E060E070E46CC0C0D0702FBED0602FB7
:104DC000BCD0502FBAD0402FB8C00E942E2600244D
:104DD0000ED1002700930401AED088EE93E0A6DF49
:104DE00011F499EE16C10197D1F70AE00F93A5D0FF
:104DF0000F910A95D9F7BEDF013069F000E4A0D029
:104E000000279ED000279CD000279AD0002798D05A
:104E100005E996D0DECFB4DF013009F01FC0CCDF4A
:104E2000513011F44A3A11F09AEEF3C0BFDF00306E
:104E300021F07CDFD9F79BEEECC0B2DF003021F02F
:104E400075DFD9F79CEEE5C0B7DF84E080930401FD
:104E500076FF1DC08CE08093040119C0A5DF0230ED
:104E600028F081E08093040101E404C082E0809393
:104E7000040109EE0F937FDF00230F9121F056DF2D
:104E8000C9F79DEEC6C084DF002309F0A2CFBAC0E7
:104E900011E0003409F415E9083409F417E807FFB4
:104EA00014C00F931F934F935F936F937F9307E704
:104EB00062DF7F916F915F914F911F91802F0F91D2
:104EC0000F77823010F0082F1EC035D02FDF31D081
:104ED0001DD011F008EE17C033D0072F31D0062FA8
:104EE0002FD0052F2DD0042F2BD0012F29D02F9379
:104EF00024E623D0189407FF05C018DF11F02A9587
:104F0000C1F798942F910093060108950F938F9302
:104F10009F9380E197E28093C20F9093C30F0DD0CF
:104F20000F3F19F001DFD9F798949F918F910F915E
:104F3000089546980895469A08950FEF01C00027F6
:104F40000EBD0DB5001FE8F70EB5089568D031F01D
:104F50004ED03CD021DF002311F091EF5AC0EDDF9D
:104F60000E3F21F0E3DED9F792EF53C092E088279D
:104F7000E4DF01930197E1F7E0DFDFDF43C04FD0CB
:104F800031F035D023D00ADF002311F095EF41C076
:104F9000BDDF11F096EF3DC00EEFD2DF0D3F11F4F3
:104FA00097EF37C092E088270191CADF0197E1F7B8
:104FB000C4DFC3DFC2DF0F7100930701053029F0A2
:104FC000009306010695086F24C01CC0409104019F
:104FD00043FD08C044275D916D917D91550F661F7B
:104FE000771F08954D915D916D917D9108958F93F7
:104FF0009F9380E29EE48093C00F9093C10F9F9196
:105000008F91089598DF99DF9927889490930501EF
:1050100008959F9390DF91DF9F910894F7CF90912F
:105020000401992392EE0895EDCF91EEF2CF91EE27
:10503000F0CFF5DF29F0DBDFA7DE002319F096EED5
:105040000C940928E0E8FFE378DF0E3F29F06EDEDC
:10505000C9F797EE0C94092890E080E16EDF019388
:105060000197E1F76ADF69DFCDDFE0E8FFE39091C8
:105070000401913081F08081807C803461F437813B
:105080003F732085118500271F5F2F4F3F4F110F62
:10509000221F331F1AC033272681237017810085F2
:1050A000007C005C1F4F2F4F818583709285990F84
:1050B000881F11F011D0F1F785818F7086500CD0C8
:1050C000F1F7012F122F232F3327E881F981019364
:1050D0001193219331930895000F111F221F331F45
:1050E0008A9508959CDF29F082DF4EDE002319F0B7
:1050F00096EE0C940928E881F9811FDF0E3F29F014
:1051000015DEC9F797EE0C94092890E080E115DFD1
:1051100001930197E1F711DF10DF74CF80DF29F0F1
:1051200066DF34DE002319F096EE0C940928E8813E
:10513000F98103DF0E3F29F0F9DDC9F797EE0C94F2
:10514000092890E080E1F9DE01930197E1F7F5DEAF
:10515000F4DE58CF64DF29F04ADF22DE002319F0A5
:1051600096EE0C94092828DEE881F9817193619309
:105170005193419347CF53DF29F039DF13DE0023EA
:1051800019F096EE0C940928E881F981D6DED5DE77
:105190000E3F29F0CBDDC1F797EE0C94092890E083
:1051A00080E4CBDE01930197E1F7C7DEC6DE2ACFAC
:1051B000ECE0F1E0ABE8B8E0992791931197E9F7BB
:1051C0000895E894843059F0863049F08E3039F0F3
:1051D00068948B3021F08C3011F093E1D0C20090B4
:1051E0000E0100F800920E0188940895ECE5F3E0BA
:1051F0004DD245555A4A09F40895C1C28A93D8DF61
:10520000FBD2C0F091E1F2DFA8F088818823F9F0A9
:10521000ECE1F3E08A9511F07096FCCF80818F77F6
:1052200021F434968081CDDF38F48881823078F0A3
:1052300093E1A5C22196A3C280930D013496A9E5FE
:10524000B1E03ED2D9D288F392E1D0DF98F38991D0
:10525000E9E6F1E01BD24050524094E1F9F4ACE6AB
:10526000B1E011D2A9E5B1E0E4D1DAD1AFE0B1E02B
:10527000F4D1A4E7B1E005D24050504019F4A2E8BF
:10528000B1E0E1D1E4E1F1E0F2D180916E018093EF
:10529000130196E1882311F0833008F070C2C2D167
:1052A00081FDC0D1A8E1B1E0D8D1AFE6B1E0EBD14A
:1052B000ACE1B1E0EED184E0F9D1B2D1AEE1B1E040
:1052C000CCD1A9E5B1E0BFD10E940332E5D1E1E73D
:1052D000F1E0D2D10050104019F4EEE7F1E0AED188
:1052E0000E94033280916B018093220195E1882313
:1052F000A9F28695F0F791F6D8D08CD1A3E2B1E06F
:10530000ACD100900E0100FA80910D01882379F450
:10531000E89486E00F5F164F2040304010F068940C
:105320008BE880930D01992790F990930E013EF43C
:10533000AAE8B1E07ED1CED0A8E1B1E08ED182E082
:1053400080932701A8E1B1E074D1AFE2B1E085D14B
:10535000A5E3B1E082D11BC227D468F080D349F421
:105360008F9390E233D48F9138F4923419F490E211
:1053700004C009C20894882708958F9381D48F911F
:1053800008F005C288270895FDD308F43EC13C9675
:1053900097D1FDC1F7D308F438C170964FD13AD1F7
:1053A0005CD1F5C1EFD350F090E2F9D538F0FA9323
:1053B000EA933FD136D608F0E9C1EFC10895E2D3B0
:1053C00030F0FA93EA93F9D308F0E0C1E6C108950A
:1053D000D9D328F0808D827009F08FEFD8C18FEF7C
:1053E000089548E006C044E004C042E002C041E045
:1053F00000C05527C7D3A8F090E2D1D590F0FA931A
:10540000EA9356F45F934F93BF93AF930AD6AF914D
:10541000BF914F915F9120F00E94B73008F0B6C164
:10542000BCC1089548E006C044E004C042E002C0A8
:1054300041E000C05527A6D3A0F090E2B0D588F097
:10544000FA93EA9356F45F934F93BF93AF93E9D5E2
:10545000AF91BF914F915F9118F040D608F096C17F
:105460009CC10895FF93EF9327D203C0FF93EF935E
:10547000D3D2AF91BF9118F4C8D0EFD0089530C304
:10548000802FC8D090911E01891B982F8395892762
:1054900090912201892311F488940895C5D005D0F4
:1054A0002ED008F4089516D0F7CFEEE1F1E0D0D079
:1054B0000E94033272F08091220180FD06C0369571
:1054C0002795179507958695F8CF0E5F1F4F2F4F9D
:1054D0003F4F0895809122010250104020403040FB
:1054E00080FD06C0000F111F221F331F8695F8CFC5
:1054F000EEE1F1E0ADD00C94FE310BD1D6DFAFE0A0
:10550000B1E0A1D000900E0100FE04C0000F111FF9
:10551000221F331F0F93012F122F232F33270E9497
:10552000FE316FD18F91E8F000900E0100FA9927BB
:10553000880F991FE80FF91F222733270191119136
:1055400036F4219131913F7032976FEF7FE03297BF
:1055500048EF5FEF0417150716F42607370710F01A
:1055600091E20DC114C151D002E0A02E442755276D
:105570006627772704C0A7E2B1E05BD0AA243F9357
:105580002F931F930F937F936F935F934F93AF92DC
:10559000B6DFAF904F915F916F917F910F911F9107
:1055A0002F913F91A3E2B1E0CD90DD90ED90FD9081
:1055B00010F4913249F5C016D106E206F30618F14F
:1055C00099278191982B8191982B2EF48191982B7A
:1055D00081918F70982B31F4A1FE0EC04F5F5F4F09
:1055E0006F4F7F4F802F912F15D09127969516F4EE
:1055F0008027880F00F7C3CF32970EF43297A7E2C7
:10560000B1E02BD0C4C092E2BAC0002711272227F4
:10561000332708950F5F1F4F2F4F3F4F0895552792
:10562000662777270C94FE3101501040204030400F
:1056300008950D911D912D913D9108950191119124
:105640002191319108954D915D916D917D910895D4
:10565000419151916191719108950D931D932D93F5
:105660003D930895019311932193319308954193AC
:1056700051936193719308952227332701911191DA
:105680000895662777274D915D9108954191519135
:1056900008954D935D930895402F512F622F732FDE
:1056A0000895005010402040304008955695479589
:1056B0008A95E1F70895440F551F8A95E1F70895FB
:1056C00084E09F9391919D938A95E1F79F9108952E
:1056D000E881F9810895A881B98118960895E88133
:1056E000F9813C960895E881F9813896BBCFE8812D
:1056F000F9813896A3CFF3DFB5CFF1DF9FCFEFDF8E
:10570000A7CFA881B9811C960895E881F981749684
:105710000895FBDF93CFE881F981808D0895E881BA
:10572000F98170960895FBDF89CFF9DF91CFF7DF1C
:1057300099CF00900E0100FA8FEF819381931EF4B0
:1057400081938FE0819342C000900E0100FA019393
:10575000119316F42193319339C0E881F981799638
:105760000895D3DF7FCFA881B981549608950F9013
:105770000F900F900F900F900F900895229608941D
:1057800090930C010895882799E4F9CF2296889484
:1057900090E0F6CF22968894089522960894089572
:1057A00080EA01C084E8E881F9819F93908D892B7C
:1057B000808F9F910895E881F9819F93908D8095C6
:1057C0008923808F9F91089588E0EDCF80916203B7
:1057D000886080936203089580915D018860809362
:1057E0005D0108950E94A62708F0D1CFC8CF0E947E
:1057F000BF2708F0CCCFC3CFA9E5B1E0EEE5F1E0DB
:10580000F1CF80E1AEE5B3E006C080E0A9E5B1E00C
:1058100002C0A9DF80E817DF0E94083231F4E89463
:105820001196EA2FFB2F1597B6CF9D91EA2FFB2FEC
:10583000792F777E872B8E93149793FF18C00F9341
:105840001F932F933F939F93AF93BF93D0DFBF914D
:10585000AF919F91A8F094FF06C0AF93BF938CD3F4
:10586000BF91AF9168F03F912F911F910F91F5DE9D
:10587000D7DFEF93FF93B6DFFF91EF916894089520
:1058800078CF49DF8670B1F44EDF00271E7F4427B2
:1058900052E0C6DE4CDF3FDF867061F43ADFF0DDB8
:1058A00020F061DFB6DF38F06FC2913221F47ADF89
:1058B00091E265CF91E063CFD2D009F065CFFA9342
:1058C000EA93A5D008F469CF83858F3099F0827C64
:1058D00089F480818E3271F0853E61F08030D1F0A4
:1058E000A881B9819C919F3311F0981303C07BE08C
:1058F000A9D0A1F0B09681E0480F25F78827581F5E
:105900005F934F930FD008F080DF4F915F91D0F6F7
:10591000903C08F492E4E991F99131CFA7E5B1E028
:10592000B8DE34CF00900E0100FC19C0AFE2B1E048
:1059300080DEA8E1B1E05F934F9385DE0E940832DC
:105940004F915F9161F4ACE1B1E06D917D914617AB
:10595000570710F091E313CF0FD05CDE18CF0CD0B7
:105960003F932F931F930F938BDD08F002CF0F917E
:105970001F912F913F910895A9E5B1E05ACE4FD0E4
:1059800008F43CC08081853E81F1803071F1B09691
:1059900081E0480FBDF78827581F5F934F93C2DF00
:1059A00008F033DF4F915F9168F7913239F55F93DB
:1059B0004F937BDD3F932F931F930F93DCDDF8F024
:1059C000B8DE6ADE0F911F912F913F917F936F9305
:1059D0005F934F9394DD0F911F912F913F9180F42E
:1059E000913281F4B1DE86D2DDCFA7E5B1E051DEA0
:1059F00020DEA3E3B1E04DDE30DEC9CEC0CEB7CEAF
:105A000093E2BDDEB8CEA881B98112960AC04427C0
:105A10005527AFE2B1E006C0A5E4B1E002C0A3E3C0
:105A2000B1E031DE06DE5A934A93EFDE50F0488152
:105A30004F70552785E03FDEE40FF51F49915991DE
:105A4000A6CEABCEFF93EF9381919D919F3311F042
:105A5000891711F47A95C1F7EF91FF910895EBE45E
:105A6000F1E08F93E89499277BE0AEF08D918A3234
:105A700019F48FE368940FC08E3239F4733011F447
:105A8000E894F3CF80E2689406C0803011F480E29D
:105A90000CC00E94AE3181938F3309F4939574301A
:105AA00009F4E8947A9509F704C080E281937A9525
:105AB000E9F780E081933C9799238F910895928D27
:105AC0009D93938D9D9300900E0100FE05C09489D7
:105AD0009D9395899D93089599279D939D930895EE
:105AE0007C96EEDDB0970895882311F49AE447CEB2
:105AF00032E0E3E6F5E0E8942081222329F4D6F0B1
:105B0000EE2EFF2E689416C0281771F1EF93FF93C5
:105B10008F9380F98F9386E03296A7E5B1E08BD31F
:105B20008F9180FB8F91FF91EF9121F411811923C7
:105B300010FF1CC03A9519F0E65EFD4FDDCFC6F4AC
:105B4000EE2DFF2D18D080839183EF93FF938F93D9
:105B500086E03296AE2FBF2FE7E5F1E086E0B1DDBB
:105B60008F91FF91EF9113CE95E409CE96E407CE85
:105B700094E405CEADDD09E1002401920A95E9F730
:105B800079970895882369F072E0E3E6F5E0908163
:105B9000981749F07A9519F0E65EFD4FF8CF93E437
:105BA000EECD9AE4ECCD089580E8ECDF28F0839503
:105BB000E1F791E48827E3CDEACD8ADD02C0E2DF98
:105BC00020F081E0F0DD6ED1D5CF08958F939F93C3
:105BD00076DE7F918F91E8F0972F6385692760FFCC
:105BE00003C0692760FD18C0FF93EF937DDFFA9330
:105BF000EA93EF91FF9168F084DD72DF6CDD5FDF87
:105C000076DD4FDD39F066DC04DE40F0BDD083DDAB
:105C1000C1CD0895C5DDFBCF98E4B1CDBECDE881FF
:105C2000F9819181917251F1E881F981808D81FD35
:105C300023C0709603DD912F802FECDC349712DDAA
:105C4000E881F9813C9604DD0E94083230F03896F4
:105C5000708172607193112704C0E881F98179968F
:105C600019279170E80FF91F8081169521F08F9305
:105C700012DE8F9108958BCD91E081CD92E67FCD9C
:105C8000FF93EF938F939F9311C0FF93EF938F93A5
:105C90009F9339D058F4923451F508C0FF93EF9395
:105CA0008F939F930CDE08F5923409F568DE00F1BE
:105CB00021D09F918F91FF93EF9316DFAF91BF910A
:105CC000C0F0FA93EA93EF91FF919F938BE0F9DC98
:105CD0009F91917090629D9312968DD214968BD263
:105CE0007BDD5EDDE991F99152CD92E348DD0894C8
:105CF00040CD41CD85EE819388279FE181939A9590
:105D0000E9F7B097089509F03ECDD9DD80F183859C
:105D10008F7D11F093E333CDFF93EF9358D0EF9144
:105D2000FF9128F1FF93EF9323D0EF91FF9185EE40
:105D3000808352DD22273327028D138D00900E01C0
:105D400000FE02C024893589ACDC79F017D0D7DB9E
:105D500080E08193819316F48193819337DDB0F7CE
:105D6000913221F4EED018F0FDC0FCC008940895E3
:105D7000E7E5F1E0A3E3B1E086E05BC2E0E1FF2705
:105D8000A7E2B1E084E055C2B8DCCFDC0E94083263
:105D9000C2F0C9F049DC732761F4622751F451273E
:105DA000569539F4AADCC1DC0E94033284E0FBDCA6
:105DB000EECC00E012E086E0FEDCE9CC84E0F3DC2F
:105DC000E6CC91E601C091E086E0EDDCD8CC72E053
:105DD000E3E6F5E08081882351F0FF93EF9332965C
:105DE000A7E5B1E086E027D2EF91FF9129F07A95FF
:105DF00029F0E65EFD4FEECF97E4C1CCC8CC89DC3C
:105E00003FDB28F088DC81FF04CDABDC91C0913210
:105E1000F9F4B1DBE8F08FEF8193819300900E01EC
:105E200000FE03C081938FE08193D0DC0F931F931A
:105E30002F933F9362DB3F912F911F910F9130F48D
:105E4000913221F4A4DC80DC45DBDCCF93E297CCFB
:105E5000089591DB30F18FEF8193819300900E01D3
:105E600000FE03C081938FE08193B0DC3F932F93BA
:105E70001F930F9338DCC7DD0F911F912F913F9136
:105E800080F0028F138F00900E0100FE02C0248B61
:105E9000358BA2DC1FDB65DCB8DB49DC80E28BDC08
:105EA0008894089538DC83FF09C02FDCAE2FBF2F04
:105EB00034968081877F81939ADCD0F02CDC86FF3A
:105EC00018C087FF02C080FF14C09DDD88F0AE2F90
:105ED000BF2F1B968C9180628C93519681E46BDC72
:105EE0000CDCBBDB1A9787D177DC3CD008F029C0EB
:105EF00008954DCCEFDA809122018F9386DC18F063
:105F000018D06ADC88948F9190F08A9529F0E9E5A1
:105F1000F1E094DB7FDBF1CF409122014A9531F033
:105F2000E9E5F1E08BDB041B80DB6FCC30CC08951E
:105F300014DC772792E080E071930197E9F7F25043
:105F400026CC80E1AEE5B3E0E2E6F3E0908193FF9A
:105F500008958193BF93AF934ADCAF91BF9108F44A
:105F600008950AC080E0A9E5B1E0EDE5F1E0908197
:105F700093FF089581933BCCE3E1F1E0819181FFB0
:105F8000089566DB56DBEA2FFB2F31960E94FE3127
:105F9000ABE2B1E062DB14972ACCE881F981092EEB
:105FA0009181902111F08894089592E6E8CBE881E0
:105FB000F98191819A7279F1E881F9818F93908DBD
:105FC00095FF06C046DF48F1B3DFE881F981908D87
:105FD000709634DBF12EE02E1DDB349743DBE88135
:105FE000F9813C9635DB401751076207730718F4B7
:105FF000349738DB92641F259860E881F9817896A0
:1060000091939F2D9170EE0DF91F8F9181931695AD
:1060100031F048DFF4CE92E6B2CB8F9108958894A8
:10602000089502DB332312F493E6A9CB19F473DB52
:1060300085FDADCB64DB0E940832C1F1A8F53F932A
:106040002F931F930F937CD05C2D6D2D7E2D4F933E
:106050006ADB76D05EDB7F936F935F9326DA5F9186
:106060006F917F915C156D057E0528F089F05C19B4
:106070006D097E0901C03BDB51506040704040F02B
:106080007F936F935F933BDA5F916F917F91A0F75E
:1060900021DA4F91C4DABDDBC8F00F911F912F9127
:1060A0003F9145DB71DE73CB91E669CB002339F676
:1060B000812F817021F6B8DAB5DF40F034DBAADA3F
:1060C00036DB9DDE20F4913011F00894089523DB37
:1060D00081FD2ECF5CCB91E260DF70F11CDB81FD96
:1060E0002CC05F934F9375D04F915F9130F166272D
:1060F00077270E94083210F4402F512F61D0415071
:106100005040B8F00F3F81F410FF0EC010DBBF937A
:10611000AF935F934F9388DD4F915F91AF91BF91A4
:1061200058F001DB1ADB03C00F5F1F4F81918D9385
:10613000E6CFFDDA4ED02BCB089534DB91E01FCBB8
:1061400080912201369527951795412F90E08695ED
:1061500030F03695279517950894991FF8CFC12EE2
:10616000D22EE32E492308959AE217DF40F128D07A
:1061700041505040B8F08D9195FD04C00F3F71F42F
:1061800010FF0CC0D4DABF93AF935F934F9314DF2B
:106190004F915F91AF91BF9190F0E9CF81930F5FE5
:1061A0001F4FE6CF11DBABDA4017510762077307C9
:1061B00018F4A1DA80E4F7DABADA0BD0E8CA089565
:1061C00087DA908DB0DAC9DA712F7170E00FF71F9E
:1061D0000895E881F981808D90DAA7DA79DA0E9452
:1061E000033228F021F08D7F808F88940895866097
:1061F000808F0894089581E0AA24BB24C82ED82E4D
:10620000E82EF82ECC0CCC0CCC0C8827B6948795B5
:10621000B69487958A29B6948795BC288D93BD92AC
:1062200084E18F0DE294EE0C881FED28ED928D93A2
:106230000895689401C0E894FA93EA93BA93AA93F4
:10624000082E8817CFB6A190BD90CFBEAB04CFB6B5
:106250008A95C9F7CFBE46F438F4802DA881B9815C
:10626000EA81FB812EDACFBEA991B991E991F9912A
:106270000895019111912191308108950F92B801F3
:10628000469F8001479F100D569F100D0F90089557
:106290000F921F922F92C801D901489F80014A9FF7
:1062A00090014B9F202C499F100D211D321D5A9F9C
:1062B000202C589F100D211D321D599F200D311D7E
:1062C000689F200D311D699F300D789F300D2F90F4
:1062D0001F900F9008950E9490310D920020D9F7E1
:1062E000089570917A00706470937A0000907A003B
:1062F00006FCFCCF70917A00706470937A00009075
:106300007A0006FCFCCF8091780090917900089586
:10631000903029F08C91880F9A95E9F78C93089525
:10632000D895319628F48F938BB783958BBF8F9137
:106330000020089591E005C092E003C094E001C000
:1063400098E0EEDF0D929A95E1F7089582E001C0A2
:1063500084E099279D938A95E9F70895813618F08E
:106360008B3708F48F7D08952E2E3F2E992781912B
:106370008D3209F093958823D1F79A95E22DF32D6C
:10638000112361F0091718F011F0101B01C0191B3F
:1063900028F021F080E28D931A95E9F780818D3203
:1063A00019F48D93319604C0222311F08BE28D9362
:1063B000091738F031F0091B21F080E38D930A951D
:1063C000E9F781918D938823E1F7332351F0EA2F88
:1063D000FB2F319633958E9182933A95E1F78EE2B9
:1063E0008C9308950F9301E00BBF0F91889408954B
:1063F0000F930027F9CF0F9302E0F6CF040F151F7C
:10640000261F371F0895041B150B260B370B089505
:1064100004171507260737070895000F111F221FBD
:10642000331F089500951095209530950F5F1F4FED
:106430002F4F3F4F0895019110810FC00E943931B5
:106440000EC00E94393110C00191108117FF05C0A4
:106450003FEF2FEF04C0008111272227332737FF9A
:1064600003C0E0DF8DE28D93CF92DF92EF92AA24FA
:10647000BB24CC24DD24EE2440E2EAE0FF2755E0F3
:1064800093E38081890F87FD9F7083FD907F891B37
:1064900081935A95A9F7C1DFAA1CBB1CCC1CDD1C3B
:1064A000EE1C4A9551F7E894EFE0FF2782910CD05B
:1064B000EB30E0F71EF068948A2D0AD088278D9380
:1064C000EF90DF90CF900895982F829501D0892F7B
:1064D0008F70805D26F0803309F4089568948D9361
:1064E000089541E003C042E001C044E0E40F882782
:1064F000F81F8291982F829506D0892F04D04A9553
:10650000C1F70C94A1328F708A3008F0895F805DEA
:106510008D93089500271127222733278D918823F3
:1065200079F07BDF7ADF79DF78DF18DF815408F4D8
:10653000895F865F080F8827181F281F381FEECF36
:10654000089588278D930895F999FECFE1BDF2BD96
:106550003196089591E001C092E07B3751F47FB706
:10656000F894F2DF8D9180BDFA9AF99A9A95C9F75D
:106570007FBF7727089591E001C092E0E5DFF89AA8
:1065800080B58D939A95D1F70895689401C0E894E9
:10659000AF93BF938D9116F0919103C00E949031FB
:1065A000902D891718F011F48823A1F7BF91AF91AE
:1065B000089500276CE8719198E00695779577FF2C
:1065C00018F477FD08F006279A95B9F78A9599F798
:1065D00008952D000000496E69742048572E2E2E14
:1065E00000004D65617375726520766F6C7461672C
:1065F000652E2E2E5B00565D0000436865636B20A0
:106600004655534520424954532E2E2E00004F4BE1
:1066100000004572726F7223000052656164696EFA
:106620006720434F4E4649472066726F6D204545AF
:1066300050524F4D2E2E2E00534420636172642021
:106640006973206E6F7420696E7365727465642E51
:106650002E2E00004572726F7220534420636172C7
:10666000642074797065202D200053656172636821
:10667000204649524D574152452E2E2E0000666944
:10668000726D776172652E6865780000536561727E
:10669000636820636F6E6669672E7232302E2E2E0D
:1066A0000000636F6E6669672E72323000005361BE
:1066B000766520636F6E6669672E72323020746F64
:1066C00020454550524F4D2E2E2E0000636F6E66B2
:1066D00069672E73323000005361766520636F6EF8
:1066E0006669672E73323020746F2053442E2E2E2D
:1066F00000005374617274696E6720706175736510
:106700002E2E2E004155544F4D41542E0000313055
:1067100030306D730000323030306D730000333034
:1067200030306D730000436F6E74726F6C20736550
:106730007474696E67732E2E2E005B496E313A00B9
:1067400020496E323A005D00436865636B20534414
:1067500020656E67696E652066696C65732E2E2EE6
:106760000000536574207661726961626C65732004
:10677000746F2064656661756C742E2E2E005374E0
:10678000617274696E67204D41494E204C4F4F50E5
:106790000000534F554E44312E5741560000534F81
:1067A000554E44322E5741560000534F554E4433F8
:1067B0002E5741560000534F554E44342E574156E4
:1067C0000000534F554E44352E5741560000534F4D
:1067D000554E44362E5741560000534F554E4437C0
:1067E0002E5741560000534F554E44382E574156B0
:1067F0000000534F554E44392E5741560000534F19
:10680000554E4431302E57415600534F554E44316A
:10681000312E57415600534F554E4431322E574179
:106820005600534F554E4431332E57415600534F67
:10683000554E4431342E57415600534F554E443136
:10684000352E57415600534F554E4431362E574141
:106850005600454E47494E4500002E574156000010
:106860005741564500003A004657575254002355A9
:106870004E535550504F52544544000052454144E8
:106880000000234F4B5245414400575249544500A4
:10689000234F4B00234F4B57525400002345525671
:1068A000455200002345524352430000454E4400E8
:1068B00023454E4400004857322E304657322E3280
:1068C00000004857322E314657322E3200004361C5
:1068D0007264202D204572726F72230043617264CE
:1068E000202D204F4B21000046696C6520537973A1
:1068F00074656D202D204572726F72230000466909
:106900006C6573797374656D202D204F4B210000E9
:00000001FF
